:104C1E007584008539D2853AD3758401853BD2855A
:104C2E003CD3E4F53AF53930007330566885668228
:104C3E00856583E0F56912821DE56C2539F539E548
:104C4E006B353AF53AA3858266858365E5656563BE
:104C5E00700AE56665647004D2668041E565641F7E
:104C6E00700CE56664FF7006756600756504305855
:104C7E002C856482856383E56AF0A38582648583CF
:104C8E0063E563641F7016E56464FF70107564005D
:104C9E007563048008853E3A853D39800030010CED
:104CAE00E539253FF539E53A3540F53A300206E566
:104CBE0033253AF53A300310E50A8536F0A4253946
:104CCE00F539E5F0353AF53A300410E5118535F051
:104CDE00A42539F539E5F0353AF53AE4F53CF53BDE
:104CEE0030080D200908853E3C853D3B8002800042
:104CFE00300A0CE53B253FF53BE53C3540F53C30B5
:104D0E000B06E533253CF53C300C10E50A8536F0F4
:104D1E00A4253BF53BE5F0353CF53C300D10E51197
:104D2E008535F0A4253BF53BE5F0353CF53C22906E
:104D3E004D80302903124D4D302A03124D5D22E570
:0E4D4E000B2509F50BE50C3508F50C93F50A5D
:104D5C0022E512250EF512E513350DF51393C31349
:104D6C00F8E5142510F514E515350FF51593C31357
:104D7C0028F511227F8285888C8F9295989B9EA115
:104D8C00A4A7AAADB0B3B6B9BBBEC1C3C6C9CBCE7E
:104D9C00D0D3D5D7D9DCDEE0E2E4E6E7E9EBEDEE03
:104DAC00F0F1F2F4F5F6F7F8F9FAFBFCFCFDFDFE78
:104DBC00FEFEFEFEFEFEFEFEFEFDFDFCFCFBFAFA18
:104DCC00F9F8F7F6F4F3F2F0EFEDECEAE8E7E5E3E7
:104DDC00E1DFDDDBD8D6D4D1CFCDCAC8C5C2C0BDCA
:104DEC00BAB7B4B2AFACA9A6A3A09D9A9794908D74
:104DFC008A8784817E7A7774716E6B6865625F5C7A
:104E0C00595653504D4A4744423F3C393734322F60
:104E1C002D2A282624211F1D1B1918161412110FB8
:104E2C000E0C0B0A0807060504040302020101001C
:104E3C000000000000000000000101020203040554
:104E4C00060708090A0B0D0E1011131516181A1C5B
:104E5C001E20222427292B2E303335383A3D404250
:104E6C0045484B4E515456595C606366696C6F7281
:104E7C0075787B7FE537F5F0753D00E53EC39456BC
:104E8C004013A4F5F0C394565007E5F02456F53EB4
:104E9C0022753EAC227456953EA4F8C39456500627
:104EAC00745698F53E22753E0022E538F5F0B401B3
:104EBC000122753F00E540C394704020200907B4DF
:104ECC00010475407022A420D20EF5F0C3947050EA
:104EDC0007E5F02470F540227540FF22C3747095ED
:104EEC0040200907B4010475407022A4F820D20BAD
:0F4EFC00C394705006747098F5402275400022E0
:107C8E00D2F4C2F5C2F675840F85F0C81253EC74A7
:107C9E0003127CDD1253DC7403127CDD1253CB1203
:107CAE0053CB7403127CDD1253CB7402127CDD12A3
:107CBE0053CB7428127D4C7406127D4C740E127DBB
:107CCE004C7401127D4C1253DC7480127D4C22C018
:107CDE0000A2E092F3A2E192F2A2E292F1A2E3926A
:107CEE00F0D2F475840F85F0C8C2F47830D8FE85D2
:107CFE00F0C87830D8FED00022C00075840FA2E400
:107D0E0092F3A2E592F2A2E692F1A2E792F0D2F4F9
:107D1E0085F0C8C2F47830D8FE85F0C87830D8FE29
:107D2E00D00022203817EF75840FD2F5C2F685F0F9
:107D3E00C8127D071253CB127CDD1253CB227584F1
:107D4E000FC2F5C2F685F0C8127D071253CB127C16
:107D5E00DD1253CB2220380DEF14A2E492E6C2E4DA
:107D6E00D2E7127D4C22740F127D4C22740D127DBF
:107D7E004C2220380E7F01127D6378107F20127DF9
:107D8E0031D8F92220380E7F11127D6378107F20B2
:067D9E00127D31D8F9222C
:10759200C2B6758400D2C2C2C6D2C6C2C4D2C5C2E5
:1075A200C330C3FD74A0F5C2C2C5C2C330C3FD8ED1
:1075B200C2C2C330C3FD8FC2C2C330C3FD8DC2C2BB
:1075C200C330C3FDD2C4C2C320C4FD1253DCD2B641
:1075D20022758400C2C3D2C530C3FD74A0F5C2C2F5
:1075E200C5C2C330C3FD8EC2C2C330C3FD8FC2C287
:1075F200C330C3FDC2C4D2C5C2C330C3FD74A1F53A
:10760200C2C2C5C2C330C3FDC2C2C2C330C3FD853C
:10761200C207D2C4C2C320C4FD22D2C2C2C6D2C6CD
:10762200D2C4C2C320C4FD22758400D2C2C2C6D253
:10763200C6C2C4D2C5C2C330C3FD74A0F5C2C2C59E
:10764200C2C330C3FD8EC2C2C330C3FD8FC2C2C328
:1076520030C3FD8C838D827B40E0A3F5C2C2C33070
:10766200C3FDDBF5D2C4C2C320C4FD1253DC2275B4
:107672008400C2C3D2C530C3FD74A0F5C2C2C5C264
:10768200C330C3FD8EC2C2C330C3FD8FC2C2C3307A
:10769200C3FDC2C4D2C5C2C330C3FD74A1F5C2C208
:1076A200C5C2C330C3FD8C838D82C2C330C3FDE526
:1076B200C2F0A31BBB01F3C2C2C2C330C3FDE5C209
:0976C200F0D2C4C2C320C4FD22B1
:050003000248D73200A5
:04000B00024C0B3266
:10553F0075FF0775FFDE75FFAD75840F75E1077594
:10554F00E20475E34475840F75A43575A50975A636
:10555F00BB75A7FF759CFF759D00759E00759FF02D
:10556F0075D8FF75E8FF75F80F75AD0F7584017568
:10557F00893075888F75840275893075888F758429
:10558F000F758A80758C67780874FF000000000023
:10559F0000000000000000D5E0F1D8EDE58C30E709
:1055AF00FB759701758A0043890475840075B710E0
:1055BF0075840F438901758D02758F01758E047483
:1055CF0080D5E0FD438902E58930E4FB75970275CC
:1055DF00840075D10775840075BB0175BA0075BC61
:1055EF00F075C70075C60075C5FF75C4FF75E881F6
:1055FF0075840275BB0475BA0075BCF175C600756C
:10560F00C4FF75E88875840075D48475840175D4DA
:10561F0084758400C2F8759A47759D1A43F8097509
:10562F00870075840075B90075A90075910075988C
:10563F005075840175989075840075C04075C300CE
:10564F0075CFF2758400758E107589217588057573
:10565F008400758A00758BE0758CF4758DE0438836
:10566F004075840075C90075CA0075CB0075CC00F4
:10567F0075CD0075840175C91875CA8075CBFB751A
:10568F00CDFB75CC80D2CA75840275C91875CAA6B0
:10569F0075CBAF75CDAF75CCA6D2CA75840075EF3B
:1056AF000275A8AC75B81D75E6B075E71775F600ED
:1056BF0075F74378A0760A76A1780A78A2760675F0
:0756CF00A8859000007F0098
:1056D6007E20E4F0A3DFFCDEFA7534327535FF7503
:1056E60036C878A0760A78A1760A78A27606D2B667
:0456F60012761C22EA
:1053610075840FD2FD2275840FC2FD2275840FD280
:10537100FC2275840FC2FC2275840FD2FED2342226
:1053810075840FC234C2FE22C29322D29322758445
:105391000FA2FA2275840FA2F92275840FA2DD22D1
:1053A100A2922275840FA2DA2275840FA2DB2275E4
:1053B100840FA2D82275840FA2D922000000000018
:1053C10000000000000000000022C000C0017904BC
:1053D10078B4D8FED9FAD001D00022C000C0E0785C
:1053E1009C7605E670FDD0E0D00022C000C0E078D8
:1053F1009C760FE670FDD0E0D00022C000C0E078BE
:105401009C7664E670FDD0E0D00022EF75F06484F4
:1054110024309000CBF0E5F0A375F00A842430F03D
:10542100A3E5F02430F022EF75F06484243090007D
:10543100CBF0E5F0A375F00A842430F0A3E5F02465
:1054410030F09000CBE0B4300B7420F0A3E0B43026
:10545100037420F022900021E0540FFFA3E0B42058
:015461000248
:105462008019540FCF75F00AA42FFFA3E0B42002D5
:105472008009540FCF75F00AA42FFF22C006C00581
:10548200C004900021E0540FFFFEA3E0B42003C348
:10549200802C540FFDCF75F00AA42FFFA3E0B42097
:1054A20003C3801A540FFCEE75F064A420D20EFEE2
:1054B200ED75F00AA42E40052C40028001D3D004E1
:1054C200D005D0062275F06484F6E5F00875F00A7E
:1054D20084F608A6F008229000D1E075F009A42F06
:1054E200FFE5F03EFE79007A537B097C008E838FC4
:1054F20082EC9389838A82F0A3A983AA820CDBEDD2
:1055020022900057E0601775F010A42FF9EE35F0E5
:10551200FA7BFFC006C00712ABECD007D0069000A2
:1055220058E0600F75F010A42FF9EE35F0FA7BFF0A
:0D55320012A61222850607222285050622F8
:1000A600564F4950205441424C4520424547494EFF
:1000B60000564F4950205441424C452057524F4E0E
:1000C600470020564F4950205441424C4520454E4A
:1000D6004420002020202020202020202020202016
:1000E6002020205245504541544552204E554D4200
:1000F6004552202020202020202020203120746FEF
:10010600203230202053495445204E554D42455209
:100116002020202020202020202020203120746F25
:1001260020393982020011010215011482020111DF
:1001360003041501632020202020202020202020D9
:1001460020202020202020202020202020202020A9
:10015600202020202020434F5552544553592042F9
:100166004545502020204354435353204F4E2048AA
:10017600414E47202020205553455220454E4142AE
:100186004C452020202020524553455256452054A8
:100196004F4E45202020204E4554574F524B204D60
:1001A6004F44452020204E4554574F524B204E5524
:1001B6004D42455220202020202020202020202093
:1001C6002020202020202020202020202020202029
:1001D6002020202020202020202020202020202019
:1001E6002020202020202020202020202020202009
:1001F60020202020202020202020202020202020F9
:1002060020313D454E202020202020202020202067
:10021600204D4F4445202020202020202020202033
:1002260020544F4E4564010011020C150001640272
:100236000011030C15000164040011040C150001E3
:1002460064080011050C15000164100011060D1557
:100256000002C8030111070A1901012020202020ED
:100266002020202020202020202020202020202088
:10027600202020202020202020202020434F5552BF
:10028600544553592042454550202020435443535A
:1002960053204F4E2048414E47202020205553459D
:1002A6005220454E41424C452020202020524553A5
:1002B6004552564520544F4E45202020204E455449
:1002C600574F524B204D4F44452020204E45545702
:1002D6004F524B204E554D42455220202020202083
:1002E6002020202020202020202020202020202008
:1002F60020202020202020202020202020202020F8
:1003060020202020202020202020202020202020E7
:1003160020202020202020202020202020202020D7
:1003260020202020202020313D454E202020202046
:10033600202020202020204D4F4445202020202012
:1003460020202020202020544F4E45640100110219
:100356000C15000164020011030C15000164040071
:1003660011040C15000164080011050C1500016448
:10037600100011060D150001C8030111070A190125
:100386000120202020202020202020202020202086
:100396002020202020202020202020202020202057
:1003A6002020434F5552544553592042454550202D
:1003B6002020205553455220454E41424C45202091
:1003C600202043524F535320544F4E45204D4F4407
:1003D600452043544353532F4443532043524F53D2
:1003E6005320204E4554574F524B204D4F444520E5
:1003F60020204E4554574F524B204E554D424552A4
:1004060020202020202020202020202020202020E6
:1004160020202020202020202020202020313D4583
:100426004E2020202020202020202020204D4F4418
:1004360045202020202020202020202020544F4E00
:100446004520202020202020202020202020202081
:10045600206401001102091500016402001103095C
:1004660015000164040011060A150001C8030111F4
:10047600070C1901012020202020202020202020E8
:100486002020202020202020202020202020202066
:1004960020202020200101010101010101010000AD
:1004A6000000000000000000000000000000000046
:1004B6000000000000000000000000000000000036
:1004C6000000000000000000000000000000000026
:1004D6000000000000000000000000000000000016
:1004E60000000000000000000000000000000020E6
:1004F60020202020202020202020202020202020F6
:100506002020202020202020202020202020200104
:1005160001010101010101010000000000000000CD
:1005260000000000000000000000000000000000C5
:1005360000000000000000000000000000000000B5
:1005460000000000000000000000000000000000A5
:100556000000000000000000000000000000000095
:1005660000000000000000000020202020202020A5
:100576002020202020202020202020202020202075
:10058600202020202020202020010101010101013E
:100596000101202020202020202020202020202093
:1005A6002020202020202020202020202020202045
:1005B60020202054454C434F2050524F4752414D26
:1005C600202020524144494F2050524F4752414D1E
:1005D60020202050484F4E452050524F4752414D03
:1005E600202020434F4D50552050524F4752414DE9
:1005F6002020202041434345535320434F44452068
:10060600202044544D462054454C434F204C4556DB
:10061600454C44544D4620524144494F204C455682
:10062600454C4245455020524144494F204C455681
:10063600454C424545502054454C434F204C455669
:10064600454C4357494420524144494F204C455656
:10065600454C564F49434520524144494F204C454D
:10066600564C564F4943452054454C434F204C4524
:10067600564C5041474520524144494F204C45561F
:10068600454C435443535320524144494F204C4513
:10069600564C44435320524144494F204C455645FD
:1006A6004C204C545220524144494F204C4556450B
:1006B6004C2052505420524144494F204C455645F7
:1006C6004C2054454C434F20524144494F204C4501
:1006D600564C524144494F2054454C434F204C45BB
:1006E600564C524144494F204C494D4954204C45A3
:1006F600564C20434F53204F5220535155454C439F
:1007060048202020434F5320504F4C4152495459C2
:100716002020434F53205452494747455220564FB5
:100726004C54434F53204143515549535420544947
:100736004D45434F532052454C454153452054495E
:100746004D452053454E534520504F4C4152495438
:10075600592053454E205452494747455220564F3B
:100766004C5453454E204143515549535420544906
:100776004D4553454E2052454C454153452054491D
:100786004D45204C545220484F4C442044454C4142
:100796005920505454205455524E4F4646205449E1
:1007A6004D4552455045415445522054494D454FBB
:1007B60055542020414E54492D4B45524348554EE1
:1007C6004B202020535155454C4348205441494C19
:1007D60020202043544353532F44435320484F4C27
:1007E600442043524F535320425553592044454CBD
:1007F600415943524F5353204255535920484F4C69
:10080600442020204C54522053594E4320424954F0
:10081600202020414456414E43454420204C4F431E
:100826004B20202020202020202020202020202097
:1008360020202020202020202020202020202020B2
:1008460020202020202020202020202020202020A2
:100856002020202020202020202020202020202092
:100866002020202020202020202020202020313D54
:10087600454E202020202020202020202052415498
:10088600494F2020202020202020202020303D43BA
:100896004F532020202020202020202020313D5092
:1008A6004F532020202020202020202020203120CF
:1008B6004D532020202020202020202020313020B1
:1008C6004D53202020202020202020203130302091
:1008D6004D5320202020202020202020202020537F
:1008E600454320202020202020202020313D534B2E
:1008F6004950202020202020202020202020202099
:1009060020202020202020202020202020202020E1
:100916002020205052494F52495459204C455645A3
:100926004C20204C545220454E434F444520504FB6
:100936004C20204C5452204445434F444520504FB0
:100946004C2020205445535420494420434F4445CD
:10095600202049444C45204D45535341474520549A
:100966004D5220202020415245412042495420200A
:100976002020204D4153544552204F5220534C4184
:1009860056452044435320454E434F444520504F3F
:100996004C2020444353204445434F444520504F68
:1009A6004C2020434F5552544553592044454C4101
:1009B600592020202048414E472054494D452020AB
:1009C6002020434152524945522044524F50204420
:1009D6004C5920204143434553532044454C4159EB
:1009E600202053544154494F4E204944204D4F44F2
:1009F600452020564F494345204F522043574944EE
:100A060020202020494420494E54455256414C202E
:100A16002020202020435749442053504545442058
:100A260020202043574944204652455155454E43C0
:100A36005920202043574944204D455353414745AB
:100A46002020205455524E5F4F4E2044454C41596C
:100A56002020205455524E5F4F46462044454C4177
:100A660059202042454550204652455155454E4352
:100A7600592052455045415445522044495341421C
:100A86004C45204155582052454C4159204D4F4424
:100A960045202043524F53532042555359204D4F22
:100AA6004445205245504541544552204741494E00
:100AB6002020202054454C434F204741494E2020BA
:100AC60020204E4554574F524B2048414E475449DB
:100AD6004D45202020202020202020204C45564512
:100AE6004C2020202020202020202020303D4E4F4A
:100AF600524D202020202020202020202020434F3F
:100B06004445202020202020202020202020415243
:100B160045412020202020202020303D4D415354A7
:100B26004552202020202020202020202020312057
:100B36004D5320202020202020202020203130202E
:100B46004D5320202020202020202020313030200E
:100B56004D532020202020202020202031302053DB
:100B66004543202020202020202020202031204DF9
:100B7600494E2020202020202020202020204D4FBC
:100B86004445202020202020202020303D564F495B
:100B960043452020202020202020202020204652AF
:100BA6004551202020202020202020202020313DBB
:100BB600454E2020414C41524D20434F554E542026
:100BC600202020524553544F524520434F554E54F2
:100BD6002020202020494E54455256414C202020AA
:100BE6002020204E4554574F524B20434F4445201A
:100BF6002020494E544552434F4E4E454354204DB6
:100C06004F444E4554574F524B20494E4143544949
:100C1600564582010011022D1500018201011103C2
:100C26002D15000182010211042D15000182010318
:100C360011052D150001780604110601190101821E
:100C4600030A11072E1500FF82030B11082E15004B
:100C5600FF82030C11092E1500FF82030D110A2EC7
:100C66001500FF82030E110B2E1500FF82030F11D4
:100C76000C2E1500FF820310110D2E1500FF8203A6
:100C860011110E2E1500FF820312110F2E1500FFF3
:100C960082031311102E1500FF82031411112E1555
:100CA60000FF82031511122E1500FF820316111381
:100CB6002E1500FF82031711142E1500FF8203184C
:100CC60011152E1500FF82011911162F150001822C
:100CD600011A11173015000182031B11182E150079
:100CE600FF82021C11193115006382021D111A328E
:100CF60015006382011E111B3015000182031F11AE
:100D06001C2E1500FF820220111D31150063820280
:100D160021111E32150063820222111F3315026350
:100D26008203231120321501FF8203241121341579
:100D360002FF820225112233150063820226112347
:100D460032150063820227112433150363820228B9
:100D56001125321500638203291126331500FA8204
:100D6600012A11273515000182012B11385415016E
:100D76000982012C11395515000182012D113A55B0
:100D860015000182032E113B561501FA82032F111D
:100D96003C5C1500FF820130113D571500018201B0
:100DA60031113E58150001820132113F55160001DE
:100DB60082013311405515000182023411415A1542
:100DC600006382023511425B1500638202361143CD
:100DD6005A15006382023711445A1500638201389E
:100DE60011455E15000182013911465F1500018229
:100DF600023A11475D15006382023B1148591504FA
:100E06006382023C114960150114BE0A3D114A561F
:100E1600110000820247114B5A15006382024811E5
:100E26004D60150114820149114E5E1500028201C2
:100E36004A114F6115000182014B11505E150004E5
:100E460082014C11515415010982014D115254155C
:100E5600010982024E11533415006382014F11625B
:100E66000115000982015011630115000982025122
:100E760011645D150163C8035211650115010182F4
:100E8600015311665E150002820354116734150082
:100E9600FF01010200000200000200000000000045
:100EA6000101013132333435361432320532FFFF57
:100EB600FF1919196464C8FF000180000A01800047
:100EC6000A1E1AB400001E1E1E00010000020100C8
:100ED6000100000A1E630A000100050520202020EB
:100EE6002020202020200A05000000010114000017
:100EF600010000000044313233343536373839309A
:100F06002A2341424344AAA3C1C2C3C4D7ABA8A95A
:100F16002A23414243363330363730363934373177
:100F2600393734343737303739373832353835345E
:100F3600383835393135393438393734313030315C
:100F4600303331303731313031313431313831327B
:100F5600333132373133313133363134313134365E
:100F66003135313135363135393136323136353143
:100F76003637313731313733313737313739313821
:100F86003331383631383931393231393631393908
:100F96003230333230363231303231383232353225
:100FA600323932333332343132353032353430300F
:100FB6003630303730313530313730323130323308
:100FC60030323530323630333130333230333630FA
:100FD60034333034373035303035313035333035E1
:100FE60034303635303731303732303733303734C6
:100FF60031313431313531313631323231323531C8
:1010060033313133323133343134313134333134B5
:101016003531353231353531353631363231363591
:10102600313732313734323035323132323134328F
:101036003233323235323236323433323434323479
:101046003532343632353132353232353532363163
:10105600323633323635323636323731323734334A
:10106600303633313133313533323533333133334F
:10107600323334333334363335313335363336342D
:101086003336353337313431313431323431333428
:101096003233343331343332343435343436343510
:1010A60032343534343535343632343634343635F4
:1010B60034363635303335303635313635323335EC
:1010C60032363533323534363536353630363631D6
:1010D60032363234363237363331363332363534C9
:1010E60036363236363437303337313237323337B5
:1010F600333137333237333437343337353441428B
:10110600434445464748494A4B4C4D4E4F50515231
:10111600535455565758595A6162636465666768F1
:10112600696A6B6C6D6E6F707172737475767778B1
:10113600797A30313233343536373839607E21406A
:101146002324255E262A28295F2D2B3D7B7D5B5D8A
:101156007C3A3B3C3E2C2E3F2F2020202020202076
:10116600202020202020474C4F42414C2020202088
:1011760020202043544353533A202020202020206F
:101186002020204443533A202020202020202020C5
:1011960020202052455045415445522020202020F1
:1011A60020205350454544204449414C494E472050
:1011B600202053504545442043414C4C494E47203E
:1011C600202020505443204E554D42455220202089
:1011D600202020564F494345204D4553534147450E
:1011E600532020564F49434520504C4159424143D4
:1011F6004B202020494E56414C49442054595045D5
:10120600202020204F5554204F462052414E47451E
:10121600202020494C4C4547414C2056414C5545D1
:1012260020204D5553542046494C4C204649454CA8
:1012360044202020494C4C4547414C20434F4445CF
:1012460020202044415441204143434550544544C5
:1012560020204C494E45204E554D4245523A2020BD
:101266002020555345522050524F4752414D4D492B
:101276004E47204C54522049443A2020202020201A
:101286002020564F494345205245434F5244494E2C
:10129600472020494C4C4547414C20454E54525915
:1012A600202020494C4C4547414C2047414E472081
:1012B6002020202020434F4D504C455445442020AB
:1012C600202020474C4F42414C20454550524F4D1F
:1012D60020202020435443535320454550524F4D20
:1012E600202020202044435320454550524F4D2076
:1012F60020202020204C545220454550524F4D204E
:101306002020204449414C494E4720454550524FE4
:101316004D202043414C4C494E4720454550524FA5
:101326004D2020202050544320454550524F4D20FB
:1013360020202052455045415445522045455052A3
:101346004F4D2020494E495449414C495A494E4730
:101356002020202052455045415445523A20202015
:101366002020202020202020202020202020202077
:101376002020202020202020202020202020202067
:101386002020202020202020202020202020202057
:101396002020202020202020202020202020202047
:1013A600202020435443535320434F444520474174
:1013B6004E472044435320434F44452047414E4720
:1013C6002020205250545220434F44452047414E3E
:1013D600472020525054522047414E47202020207B
:0213E6002020C5
:107DA40030363230350912B22F12514602AAE91286
:107DB400B4AB128ABC12A13112A18D12B3A53050FA
:107DC40005C250123D28129FB9E490022DF0900292
:107DD4002EF0C2362230372E30350512B25F803293
:107DE40012B4AB128ABC12A13112A18D12B3A51226
:107DF4009FB9305005C250123D28E490022DF090F6
:107E0400022EF0C23722203803027EA83035061233
:107E14005BEE02514630511A12B4AB128ABC12A165
:107E24003112A18D12B3A5129FB9305005C2501260
:107E34003D28E490022DF090022EF0C2382059FD26
:107E4400900264747EF0D2592059FD9002647450FB
:107E5400F0D2592059FD9000D6E075F00A844430E0
:107E6400900264F0D2592059FD9000D6E075F00AD2
:107E740084E5F04430900264F0D2592059FD900218
:107E840064305105745DF08003745BF0D25920595D
:107E9400FD900264740DF0D2592059FD900264746F
:057EA4000AF0D2592292
:10514600900013E07012900014E0D394004009C25E
:1051560036C237C238C23522900014E0127F7E5222
:105166007700527A01527D0252800352830452859F
:1051760005528706528907528C08528F0A52920BA3
:1051860052950F529810529B11529E1452A11552CD
:10519600A41652A71952AA1A52AD1B52B01E52B3E8
:1051A6001F52B62352B92452BC2852BF2952C22DCF
:1051B60052C52E52C82F52CB3052CE3252D1335214
:1051C600D33452D63552D93752DC3852DF6452E2E4
:1051D6006552E56652E86752EB6E52ED6F532F70DB
:1051E60052EF7152F17852F379532F7A52F57B527E
:1051F600F78252F983532F8452FB8552FE8C53015A
:105206008D532F8E53038F530696530997532F981A
:10521600530B99530EA05311A1532FA25314A3530A
:1052260017AA5319AB532FAC531BAD531EB45321BE
:10523600B5532FB65324B75326BE5329BF532CC09C
:10524600532FC15331C25334C85337C9532FCA538E
:105256003DCB5340F05343F15346F25349FA534C76
:10526600FB534FFC5352FD5355FE5358FF0000535A
:105276005B02B74302B59302A35102B4D380048004
:1052860002800002A6E602625102AEE902B03202D4
:10529600AB29028B6702B06502AB68028A0F02B0C7
:1052A6009802ABA702859E02B0CB02A3FD02B0FE18
:1052B60002A45202B13102A4A702B16402B2ED0205
:1052C600AE7702A73012A29F02A2458000029B354C
:1052D60002A8DA0299E402A0D502A01A02A8960250
:1052E600AF91025F248039804880408033801C80E3
:1052F6003A8005803C0266C00287298034026557E1
:105306000293108006026DB002895F029AC602609F
:10531600BB800D801C0263E5028F1B029D4E800B35
:1053260002942202A64A028CB3800902824E028DA2
:10533600EB02971E02AD51029A5602B31B0283FE80
:1053460002B766029CE402001202006A02007602BC
:0B5356008E84020077E4900014F02227
:10B74300E4900016F0900013741EF0900014E004CF
:02B75300F022E2
:10B59300127D80127D927BFF7A12796812ABEC7F69
:10B5A30011127D63C23CC239E4900016F09000147E
:04B5B300E004F0229E
:10A35100303952900015E0FFC239BF2A079000142E
:10A36100E004F022BF5D0AC235E4900014F0D2513E
:10A3710022BF5B0AC235E4900014F0C25122BF2310
:10A38100247F23127D31900016E004F0E0C3940491
:10A39100400DC235E4900014F0127D80027D929050
:05A3A10000147402F03D
:01A3A6002294
:10B4D3007BFF7A12796812ABEC127D927F11127D99
:10B4E3006312002EE4900050F07F2A127D31C23C9B
:07B4F300900014E004F022B8
:10A6E600303946900015E0F517C239E517642A603F
:10A6F60038AF1712B7A65022AF17127D319000500F
:10A70600E02417F582E43400F583E517F090005055
:10A71600E004F0900014E004F0227BFF7A127998AE
:09A7260012ABEC90001474FAF07F
:01A72F002207
:106251002039030263E4900015E0FFC239BF2A0729
:106261009000147403F022EF642360030263D512DB
:106271007D31900018E06439707CA3E06439707658
:10628100A3E064397070D23D900017E0FFB431088B
:10629100E490004AF0026327EFB43208E490004B27
:1062A100F002633FEFB433028043900017E0FFB484
:1062B1003408E490004CF002636DEFB43508E490CB
:1062C100004DF0026383EFB43608E490004EF00213
:1062D1006399EFB437028015900017E0FFB43809D5
:1062E1009000497401F00263CEEFB4390B7BFF7A61
:1062F1001279A80263DBC23D900017E0FFB43016AB
:10630100A3E0B43011A3E0B4300CA3E0B4300790A3
:106311000014740AF022EFB43113900018E0B43085
:106321000C12B5DA5007900014740FF02290001788
:10633100E0B43211A3E0B4300C12B5DA500790008A
:10634100147414F022900017E0B43311A3E0B430B8
:106351000C12B5DA50079000147419F0229000174E
:10636100E0B4340FA3E0B4300A12B6B5900014744F
:106371001EF022900017E0B4350FA3E0B4300A12EA
:10638100B6CA9000147423F022900017E0B4360FBF
:10639100A3E0B4300A12B6DF9000147428F0229002
:1063A1000017E0B43716A3E0B43011A3E0B4300C09
:1063B100A3E0B43007900014742DF022900017E090
:1063C100B43811A3E0B4300C12B5DA5007900014C0
:1063D1007437F0227BFF7A12799812ABEC9000149B
:0363E10074FAF05B
:0163E4002296
:10AEE90090004F740BF09000507407F0E490005CF0
:10AEF900F0A3F090005E7402F0E490005FF0A3F01C
:10AF09007BFF7A11796812ABEC12A60C7F1E127DB9
:08AF1900639000147432F02271
:10B03200129887D39000D1E094019000D0E0940060
:10B04200400A12ABE690001474FAF0227E017F29C6
:10B052001254D97E007FD9125503900053E090001C
:03B0620014F022C5
:10AB29007BFF7A11799812ABEC7BFF7A1179781255
:10AB3900A6127F0E127D63900019E0FF127D3190FD
:10AB4900001AE0FF127D317F1A127D6390004F7465
:0FAB590010F09000507404F09000147432F02249
:108B6700303E079000147403F02290001BE0643934
:108B77007041A3E06439703BA3E06439703590001D
:108B87004F7411F09000507407F07BFF7A1379C887
:108B970012ABECD23D900049E075F099A42469FE30
:108BA700E5F034FF90005CF0CE12A5FD7F1E127D2C
:108BB70063804212A60C7F1E127D631298FC503C04
:108BC70090004F7411F09000507407F0900049E046
:108BD70075F099A42469FEE5F034FF90005CF0A3DA
:108BE700CEF090005E7403F090004AE0FF90005FC3
:108BF700E4F0A3EFF09000147432F02212ABE69089
:068C0700001474FAF022D3
:10B06500129887D39000D1E094059000D0E0940029
:10B07500400A12ABE690001474FAF0227E027F2B90
:10B085001254D97E017F3B125503900053E0900086
:03B0950014F02292
:10AB68007BFF7A11799812ABEC7BFF7A1179881206
:10AB7800A6127F0E127D63900019E0FF127D3190BE
:10AB8800001AE0FF127D317F1A127D6390004F7426
:0FAB980015F09000507404F09000147432F02205
:108A0F00303E079000147403F02290001BE064398D
:108A1F007042A3E06439703CA3E064397036900073
:108A2F004F7416F09000507407F07BFF7A1379C8DB
:108A3F0012ABECD23D900049E0FF7E007C017D50EF
:108A4F00127F01EF24A6FFEE340A12A5F87F1E1243
:108A5F007D63804812A60C7F1E127D63129797507C
:108A6F004290004F7416F09000507407F090004938
:108A7F00E0FF7E007C017D50127F01EF24A6FFEE08
:108A8F00340A90005CF0A3EFF090005E7403F09056
:108A9F00004BE0FF90005FE4F0A3EFF09000147440
:0D8AAF0032F02212ABE690001474FAF022AF
:10B09800129887D39000D1E094059000D0E09400F6
:10B0A800400A12ABE690001474FAF0227E037F5136
:10B0B8001254D97E027F61125503900053E090002C
:03B0C80014F0225F
:10ABA7007BFF7A11799812ABEC7BFF7A12797812D6
:10ABB700A6127F0E127D63900019E0FF127D31907F
:10ABC700001AE0FF127D317F1A127D6390004F74E7
:0FABD7001AF09000507404F09000147432F022C1
:10859E00303E079000147403F02290001BE0643903
:1085AE007042A3E06439703CA3E0643970369000E9
:1085BE004F741BF09000507407F07BFF7A1379C84C
:1085CE0012ABECD23D900049E0FF7E007C027DEEC6
:1085DE00127F01EF2448FFEE342312A5F87F1E12FE
:1085EE007D63806512A60C7F1E127D63129E88909D
:1085FE0000D2E0FEA3E0FFD39400EE94004051EFD2
:10860E0094FBEE9400504990004F741BF090005074
:10861E007407F0900049E0FF7E007C027DEE127F31
:10862E0001EF2448FFEE342390005CF0A3EFF090AE
:10863E00005E7403F09000D3E024FFFE9000D2E0C1
:10864E0034FF90005FF0A3CEF09000147432F0224D
:0A865E0012ABE690001474FAF0224B
:10B0CB00129887D39000D1E094039000D0E09400C5
:10B0DB00400A12ABE690001474FAF0227E047F57FC
:10B0EB001254D97E037F87125503900053E09000D2
:03B0FB0014F0222C
:10A3FD0090004F741FF09000507407F090005C7443
:10A40D0060F0A374CEF0E490005EF090004CE0FF9D
:10A41D0090005FE4F0A3EFF07BFF7A1179A812AB07
:10A42D00EC12A60C7F0F127D63900019E0FF127DD8
:10A43D003190001AE0FF127D317F1E127D63900076
:05A44D00147432F0223E
:10B0FE00129887D39000D1E094FF9000D0E094FF97
:10B10E00400A12ABE690001474FAF0227E047F9B84
:10B11E001254D97E047F7B125503900053E09000A9
:03B12E0014F022F8
:10A4520090004F7424F09000507407F090005C74E8
:10A4620060F0A374CEF0E490005EF090004DE0FF47
:10A4720090005FE4F0A3EFF07BFF7A1179B812ABA2
:10A48200EC12A60C7F0F127D63900019E0FF127D83
:10A492003190001AE0FF127D317F1E127D63900021
:05A4A200147432F022E9
:10B13100129887D39000D1E094FF9000D0E094FF63
:10B14100400A12ABE690001474FAF0227E057F15D6
:10B151001254D97E047FF5125503900053E09000FC
:03B1610014F022C5
:10A4A70090004F7429F09000507407F090005C748E
:10A4B70060F0A374CEF0E490005EF090004EE0FFF1
:10A4C70090005FE4F0A3EFF07BFF7A1179C812AB3D
:10A4D700EC12A60C7F0D127D63900019E0FF127D30
:10A4E7003190001AE0FF127D317F1E127D639000CC
:05A4F700147432F02294
:10B16400129887D39000D1E094FF9000D0E094FF30
:10B17400400A12ABE690001474FAF0227E057F8F29
:10B184001254D97E057F6F125503900053E090004E
:03B1940014F02292
:10B2ED003038079000147401F02290004F742EF046
:10B2FD009000507407F07BFF7A1179D812ABEC12E5
:0EB30D00A60C7F1E127D639000147432F02295
:10AE7700303E07900014742FF02290001EE06438D3
:10AE87006005A3E0B4390A12ABE690001474FAF037
:10AE9700227BFF7A12798812ABEC90001EE0540FE8
:09AEA700F55A9000147430F022F9
:10A7300090001EE064386005A3E0B4390A12ABE66D
:10A7400090001474FAF0227BFF7A1179E812ABECD6
:10A7500090001EE0540FF55AD202D20B9000F8E0A0
:10A76000F534125D8A7BFF7A1279B812ABECC20223
:09A77000C20B90001474FEF022EB
:10A29F0090001EE0540FF55A303602D200125D9C2A
:10A2AF0090026C7414F0C26730361B202704E5420D
:10A2BF0070F9125D93C2007BFF7A1279B812ABEC82
:10A2CF0090001474FEF030371F20250AE542600617
:10A2DF0012B71C3067F3125D937BFF7A1279B812B5
:08A2EF00ABEC90001474FEF0CA
:01A2F7002244
:10A24500303956900015E0FF900048F0C239127D74
:10A2550031900048E0FF12B7A65021900048E0FF7A
:10A26500900050E02417F582E43400F583EFF09078
:10A275000050E004F0900014E004F022900048E063
:10A28500B42A079000147403F0227BFF7A127998A0
:0AA2950012ABEC90001474FAF022F2
:109B350030396A900015E0FF900048F0C239127D77
:109B450031900048E0FFB42A0B90004FE0900014DC
:109B5500F0D23E22EFB4230B90004FE0900014F0BA
:109B6500C23E22900048E0FF12B7A650219000485F
:109B7500E0FF900050E02417F582E43400F583EF10
:109B8500F0900050E004F0900014E004F0227BFF18
:0E9B95007A12799812ABEC90001474FAF02258
:10A8DA0030393F900015E0FF900048F0127D31C2F8
:10A8EA0039900048E0FFB42A0B90004FE090001422
:10A8FA00F0D23E22EFB4230B90004FE0900014F008
:10A90A00C23E227BFF7A12799812ABEC9000147443
:03A91A00FAF0222E
:1099E40090004F7438F09000507407F090005C744D
:1099F40060F0A374CEF090005E7456F0303D15E430
:109A040090005FF0A3F07BFF7A1379D812ABEC12CD
:109A1400A60C8032900049E024FFFEE434FF90005D
:109A24005FF0A3CEF07BFF7A13795812ABEC12A649
:109A34000C7F0C127D63900019E0FF127D319000C1
:109A44001AE0FF127D317F1E127D63900014743280
:029A5400F022FE
:10A0D500129887D39000D1E094469000D0E0940088
:10A0E500400A12ABE690001474FAF0227E0C7F1839
:10A0F5001254D9900057E0FF601175F010A4249810
:10A10500F9740535F0FA7BFF12ABEC900058E0FFCF
:10A11500601175F010A42498F9740535F0FA7BFFE9
:0CA1250012A612900053E0900014F022EB
:10A01A00900056E0FF7003303E45127D6312B4573C
:10A02A001275D3900170EFF0900054E05F900170C8
:10A03A00F060047F3180027F30127D31303E20C2D1
:10A04A003E900170E090003760057431F08003742F
:10A05A0030F09000477401F090001474F0F02290F0
:0EA06A000059E0FF127D63900014E004F02224
:10A89600303940900015E0FF900048F0C239127D33
:10A8A60031900048E0FFB42A079000147403F022A8
:10A8B60012B7A6500F900048E0900021F0900014C7
:10A8C600E004F0227BFF7A12799812ABEC90001428
:04A8D60074FAF022FE
:10AF9100303932900015E0FF900048F0C239BF2AE5
:10AFA100079000147403F022900048E0B423079046
:10AFB1000014E004F0227BFF7A12799812ABEC9036
:06AFC100001474FAF022F6
:105F2400203D03025FB6900017E064386003025F0F
:105F3400B690005FF0A3F012B4579000D4EEF0A333
:105F4400EFF01275D3900170EFF09000517401F0EE
:105F5400900021E0B4311C900170E0FF900054E007
:105F6400FEEF4E900170F0FD9000D4E0FEA3E0FF40
:105F7400127592900021E0B43018900054E0F4FFC0
:105F8400900170E05FF0FD9000D4E0FEA3E0FF120A
:105F94007592900060E004F0700690005FE004F0F9
:105FA400C3900060E0941490005FE0940040880285
:105FB40060AB203D03026047900017E06433600348
:105FC40002604790005FF0A3F012B4579000D4EE43
:105FD400F0A3EFF01275D3900170EFF090005174BC
:105FE40001F0900021E0B4311C900170E0FF9000BA
:105FF40054E0FEEF4E900170F0FD9000D4E0FEA35B
:10600400E0FF127592900021E0B43018900054E043
:10601400F4FF900170E05FF0FD9000D4E0FEA3E097
:10602400FF127592900060E004F0700690005FE04B
:1060340004F0C3900060E094FA90005FE0940040A4
:1060440088805D12B4579000D4EEF0A3EFF012757F
:10605400D3900170EFF09000517401F0900021E0B2
:10606400B4311E900170E0FF900054E0FEEF4E90BA
:106074000170F0FD9000D4E0FEA3E0FF1275928061
:106084001F900021E0B4301F900054E0F4FF900111
:1060940070E05FF0FD9000D4E0FEA3E0FF12759283
:1060A40090001474FEF0227BFF7A12799812ABEC04
:0760B40090001474FAF022C1
:10942200900056E0FF7003303E68127D6312B4571D
:109432009000D4EEF0A3EFF0E4900170F0900054AD
:10944200E0FF900170E0C39F50349000D4E475F0C7
:1094520001127F68AFF0FE1275D3900171E4F0A3A0
:10946200EFF0E0FF900170E02437F582E43400F57C
:1094720083EFF0127D31900170E004F080BF303E46
:1094820011C23E900054E0900047F090001474F036
:10949200F022900050740AF0900059E0FF127D63B0
:0794A200900014E004F02229
:10971E00303975900015E0FF900048F0C239127D87
:10972E0031900048E0FFB42A079000147403F02231
:10973E00EFB42308900014E004F0803912B7A6505D
:10974E0038900048E0FF900050E0FE04F074172EB1
:10975E00F582E43400F583EFF0900054E02409FF25
:10976E00E433FE900050E0D39FEE6480F87480984E
:10977E004016900014E004F0227BFF7A12799812C2
:09978E00ABEC90001474FAF02217
:10AD5100303937900015E0FF900048F0C239127D7C
:10AD610031900048E0FFB42A079000147403F022E8
:10AD7100EFB42307900014E004F0227BFF7A1279EC
:0BAD81009812ABEC90001474FAF02262
:10824E00303D7B900017E06433707390005FF0A3B5
:10825E00F012B4579000D4EEF0A3EFF090005074EB
:10826E000AF0E4900170F0900054E0FF900170E08D
:10827E00C39F502B9000D4E475F001127F68AFF0CD
:10828E00FE900050E0FD04F074172DF582E43400EA
:10829E00F583E0FD127592900170E004F080C890B5
:1082AE000060E004F0700690005FE004F0C3900000
:1082BE0060E094FA90005FE094004095804E12B416
:1082CE00579000D4EEF0A3EFF0900050740AF0E453
:1082DE00900170F0900054E0FF900170E0C39F5049
:1082EE002B9000D4E475F001127F68AFF0FE900081
:1082FE0050E0FD04F074172DF582E43400F583E0B0
:10830E00FD127592900170E004F080C87BFF7A1226
:0C831E0079B812ABEC90001474FEF02251
:109AC60030396B900015E0FF900048F0C239127DE6
:109AD60031900048E0FFB42A079000147403F02286
:109AE60012B7A6501A900048E0FF900050E0FE041E
:109AF600F074172EF582E43400F583EFF080107BC6
:109B0600FF7A12799812ABEC90001474FAF0229056
:109B16000054E02409FFE433FE900050E0D39FEEAA
:0F9B26006480F87480984006900014E004F022E8
:10872900900056E0FF7006203E030287D4127D6355
:1087390012B4579000D4EEF0A3EFF01275D312548F
:1087490028900054E0B401109000CDE0FF127D3173
:108759009000CDE0900037F0900054E0B4022090F2
:1087690000CCE0FF127D319000CDE0FF127D319009
:1087790000CCE0900037F09000CDE0900038F09008
:108789000054E0640370309000CBE0FF127D31901B
:1087990000CCE0FF127D319000CDE0FF127D3190D9
:1087A90000CBE0900037F09000CCE0900038F090DA
:1087B90000CDE0900039F0303E11C23E900054E007
:1087C900900047F090001474F0F022900059E0FFF7
:1087D900127D63900050740AF0900014E004F022B6
:1066C00012547E500302681C125456900170EFF071
:1066D00090005AE0FEEFC39E500302681CA3E0FF47
:1066E000900170E0D39F400302681C303D41900050
:1066F00017E06431703990005FF0A3F012B4579046
:1067000000D4EEF0A3EFF0900170E0FD12759290CE
:106710000060E004F0700690005FE004F0C39000B9
:1067200060E0943390005FE0940040D002680C3049
:106730003D41900017E06432703990005FF0A3F0A3
:1067400012B4579000D4EEF0A3EFF0900170E0FD8A
:10675000127592900060E004F0700690005FE00413
:10676000F0C3900060E0947090005FE0940040D02F
:1067700002680C303D40900017E0643370389000A0
:106780005FF0A3F012B4579000D4EEF0A3EFF090B6
:106790000170E0FD127592900060E004F0700690C8
:1067A000005FE004F0C3900060E094FA90005FE0C6
:1067B000940040D08056303D40900017E06438701F
:1067C0003890005FF0A3F012B4579000D4EEF0A31D
:1067D000EFF0900170E0FD127592900060E004F01F
:1067E000700690005FE004F0C3900060E0941490A5
:1067F000005FE0940040D0801312B4579000D4EEB4
:10680000F0A3EFF0900170E0FD1275927BFF7A1219
:1068100079B812ABEC90001474FEF02212ABE69043
:06682000001474FAF022DE
:1065570012547E50030266B6125456900170EFF043
:1065670090005AE0FEEFC39E400BA3E0FF9001703E
:10657700E0D39F4009900170E060030266B6303DAA
:1065870041900017E06431703990005FF0A3F0127A
:10659700B4579000D4EEF0A3EFF0900170E0FD1235
:1065A7007592900060E004F0700690005FE004F0E0
:1065B700C3900060E0943390005FE0940040D00205
:1065C70066A6303D41900017E06432703990005F55
:1065D700F0A3F012B4579000D4EEF0A3EFF09001BF
:1065E70070E0FD127592900060E004F07006900074
:1065F7005FE004F0C3900060E0947090005FE09467
:106607000040D00266A6303D40900017E06433702A
:106617003890005FF0A3F012B4579000D4EEF0A3C7
:10662700EFF0900170E0FD127592900060E004F0C9
:10663700700690005FE004F0C3900060E094FA9069
:10664700005FE0940040D08056303D40900017E056
:106657006438703890005FF0A3F012B4579000D4FC
:10666700EEF0A3EFF0900170E0FD127592900060DC
:10667700E004F0700690005FE004F0C3900060E073
:10668700941490005FE0940040D0801312B45790A8
:1066970000D4EEF0A3EFF0900170E0FD1275927B4D
:1066A700FF7A1279B812ABEC90001474FEF0221244
:0966B700ABE690001474FAF02225
:10931000900056E0FF7003303E6A127D6312B4572E
:109320009000D4EEF0A3EFF01275D3900170EFF03F
:109330001294A9E4900170F0900170E0FFC39404CE
:109340005030E0FE24CBF582E43400F583E0FD7478
:10935000372EF582E43400F583EDF074CB2FF582DF
:10936000E43400F583E0FF127D31900170E004F0F9
:1093700080C6303E0FC23E9000477403F090001448
:1093800074F0F022900059E0FF127D639000507459
:099390000AF0900014E004F02240
:106DB0007F0A127A47900170EFF07003026EE7309D
:106DC0003D42900017E06431703A90005FF0A3F00C
:106DD00012B4579000D4EEF0A3EFF0900170E014DD
:106DE000FD127592900060E004F0700690005FE084
:106DF00004F0C3900060E0943390005FE0940040A2
:106E0000CF026ECF303D42900017E06432703A906E
:106E1000005FF0A3F012B4579000D4EEF0A3EFF0AF
:106E2000900170E014FD127592900060E004F07023
:106E30000690005FE004F0C3900060E09470900062
:106E40005FE0940040CF026ECF303D41900017E0EC
:106E50006433703990005FF0A3F012B4579000D4FF
:106E6000EEF0A3EFF0900170E014FD127592900027
:106E700060E004F0700690005FE004F0C3900060F2
:106E8000E094FA90005FE0940040CF8042303D43B0
:106E9000900017E06438703B90005FF0A3F012B4EC
:106EA000579000D4EEF0A3EFF0900170E014FD12C3
:106EB0007592900060E004F0700690005FE004F0CE
:106EC000C3900060E0941490005FE0940040CF7B9A
:106ED000FF801C12B4579000D4EEF0A3EFF09001A5
:106EE00070E014FD127592900170E07BFF600E7AE5
:106EF0001279B812ABEC90001474FEF0227A127979
:0B6F00003812ABEC90001474FAF02281
:10895F00900056E0FF7006203E030289FA127D63F5
:10896F0012B4579000D4EEF0A3EFF01275D3125457
:10897F00289000D4E475F001127F68AFF0FE1275F5
:10898F00D312540C9000CCE0FF900037F0A3F012FC
:10899F007D319000CDE0FF127D319000D4E475F071
:1089AF0001127F68AFF0FE1275D312540C9000CBFA
:1089BF00E0FF900039F09000CCE090003AF090008A
:1089CF00CDE090003BF0127D319000CCE0FF127DA6
:1089DF00319000CDE0FF127D31303E0FC23E90004E
:1089EF00477405F090001474F0F022900059E0FFE6
:1089FF00127D63900050740AF0900014E004F0228E
:1060BB00900021E0540F75F00AA4FFA3E0540F2FBA
:1060CB00900170F0FD900024E0540F75F00AA4FBD2
:1060DB00AAF0900023E0540F75F064A42BFFE5F0B9
:1060EB003AFE900025E0540F7A002FFFEA3E900114
:1060FB0074F0A3EFF0EDC394014022900170E0D354
:10610B0094145019900174E0FEA3E0FFC39401EEC8
:10611B0094004009D3EF94FAEE9400400A12ABE6D8
:10612B0090001474FAF022303D5E900017E0643159
:10613B00705690005FF0A3F012B4579000D4EEF0BD
:10614B00A3EFF09000D4E475F001127F68AFF0FE7E
:10615B00900170E0FD1275929000D4E0FEA3E0FF79
:10616B00900175E0FD127592900060E004F07006EE
:10617B0090005FE004F0C3900060E0943390005F08
:10618B00E0940040B3026241303D5D900017E06443
:10619B0032705590005FF0A3F012B4579000D4EE1C
:1061AB00F0A3EFF09000D4E475F001127F68AFF02C
:1061BB00FE900170E0FD1275929000D4E0FEA3E01A
:1061CB00FF900175E0FD127592900060E004F07095
:1061DB000690005FE004F0C3900060E094709000C4
:1061EB005FE0940040B3804E12B4579000D4EEF0B1
:1061FB00A3EFF09000D4E475F001127F68AFF0FECE
:10620B00900170E0FD127592900024E0540F75F030
:10621B000AA4FF900023E0540F75F064A42FFF90A5
:10622B000025E0540F2F900170F0FD9000D4E0FE9C
:10623B00A3E0FF1275927BFF7A1279B812ABEC9048
:06624B00001474FEF022B5
:1063E5007F0D127A47EF701A900024E0B43010A3A5
:1063F500E0B4300BA3E0B43006A3E06430600302E0
:1064050064EF900028E0FF64306004EFB4350E902F
:106415000029E0540FD3940540030264EF9000284F
:10642500E0FF64316004EFB4361190002DE0B42034
:106435000790002CE0B420030264EF900028E0FFF1
:1064450064326004EFB4371190002CE0B42007905B
:10645500002BE0B420030264EF900028E0FF6433D2
:106465006004EFB43809900029E0B42002807B90E5
:106475000028E0FF64346005EF64397077900029E7
:10648500E0540F75F00AA4FFA3E0540F2F9001709C
:10649500F0FD90002CE0540F75F00AA4FBAAF090D3
:1064A500002BE0540F75F064A42BFFE5F03AFE9045
:1064B500002DE0540F7A002FFFEA3E900174F0A3FF
:1064C500EFF0EDC394014022900170E0D394145095
:1064D50019900174E0FEA3E0FFC39401EE9400401F
:1064E50009D3EF94FAEE9400400A12ABE69000143B
:1064F50074FAF02212B4579000D4EEF0A3EFF090A6
:106505000050740AF0E4900170F0900054E0FF90A0
:106515000170E0C39F502B9000D4E475F001127F09
:1065250068AFF0FE900050E0FD04F074172DF58281
:10653500E43400F583E0FD127592900170E004F0FB
:1065450080C87BFF7A1279B812ABEC90001474FE08
:02655500F02232
:108F1B00900056E0FF7003303E73127D6312B4571E
:108F2B009000D4EEF0A3EFF0E4900170F0900054B9
:108F3B00E0FF900170E0C39F503F9000D4E475F0C8
:108F4B0001127F68AFF0FE1275D3900171E4F0A3AC
:108F5B00EFF0E0FF900170E02437F582E43400F588
:108F6B0083EFF0900171E0FEA3E0FF1275D3127D49
:108F7B0031900170E004F080B4303E11C23E90009D
:108F8B0054E0900047F090001474F0F022900059D8
:108F9B00E0FF127D63900050740AF0D23C900014F5
:048FAB00E004F022CC
:109D4E00303965900015E0FF900048F0C239BF2A07
:109D5E00079000147403F022900048E0FFB423082B
:109D6E00900014E004F0803DEF547FFF127D31909F
:109D7E000048E0547FFF900050E0FE04F074172E70
:109D8E00F582E43400F583EFF0900054E02409FFEF
:109D9E00E433FE900050E0D39FEE6480F874809818
:099DAE004006900014E004F022CC
:10A64A0030394B900015E0FF900048F0C239BF2A1C
:10A65A00079000147403F022900048E0FFB4230B23
:10A66A00900014E004F0E004F0801012B7A6500F36
:10A67A00900048E0900052F0900014E004F0227B31
:0FA68A00FF7A12799812ABEC90001474FAF02258
:108CB300203903028D4F900015E0FF900048F0C269
:108CC30039BF2A079000147403F022900048E0FF94
:108CD300B4230A900014E004F0E004F02212B7A6D3
:108CE300505B900052E0540F75F00AA4FF900048C7
:108CF300E0540F2FF0E090110493FF900048F0121E
:108D03007D31900048E0FF900050E0FE04F07417BE
:108D13002EF582E43400F583EFF0900054E024094B
:108D2300FFE433FE900050E0D39FEE6480F874803C
:108D330098900014E0400304F02214F0227BFF7AA1
:0D8D430012799812ABEC90001474FAF02233
:108DEB00900056E0FF7003303E7A127D6312B45749
:108DFB009000D4EEF0A3EFF01275D3C0079000D51E
:108E0B00E02401FF9000D4E03400FE1275D3AD07CF
:108E1B00D00712553B900061EEF0A3EFF012A6992C
:108E2B009000CBE0FF127D319000CCE0FF127D3142
:108E3B009000CDE0FF127D319000CBE0900037F039
:108E4B009000CCE0900038F09000CDE0900039F02D
:108E5B00303E11C23E900054E0900047F090001459
:108E6B0074F0F022900059E0FF127D639000507473
:098E7B000AF0900014E004F0225A
:109A560012B1FD900171EEF0A3EFF0D394E7EE940E
:109A6600035053D25012B4579000D4EEF0A3EFF047
:109A7600900171E0FEA3E0FF12553AAD079000D4C5
:109A8600E0FEA3E0FF127592900171E0FEA3E0FFF5
:109A9600125536AD079000D5E02401FF9000D4E0C2
:109AA6003400FE1275927BFF7A1279B812ABEC90F5
:109AB600001474FEF02212ABE690001474FAF02241
:10B31B0030360B900120E0900006F012536130386C
:10B32B0005E4900006F030370E90000630340574BB
:0EB33B000AF080037428F0900014E004F02261
:1083FE00900006E060030284CF1277F930383E20F9
:10840E0059FD900264747EF0D2592059FD90026499
:10841E007450F0D2592059FD9000D6E075F00A84C0
:10842E004430900264F0D2592059FD9000D6E07588
:10843E00F00A84E5F04430900264F0D25990005373
:10844E00E0127F7E847764847C6E847C78847C8268
:10845E00847C8C847E968483A08488AA848DB48444
:10846E0092BE847CC80000849A12B4FA801E8019D1
:10847E0012AC61801712AC9D8012120078800D1222
:10848E000079800812AA69800312A5A530360F90D4
:10849E00010CE0900001F0900014E004F02230385E
:1084AE001A2059FD900264740DF0D2592059FD9096
:1084BE000264740AF0D259C238C2359000147401A5
:0284CE00F0229A
:10B76600900001E070091253679000147401F022F2
:109CE400303611900120E0900006F012536190008C
:109CF40006E070FA30370C9000067405F090000608
:109D0400E070FAE4900170F030370C12B82112536D
:109D1400FC12B84B1253FC30360C12B82C1253FC04
:109D240012B84B1253FC900170E004F0E0C39405A8
:109D340040D630360E90010CE0900001F090000106
:0A9D4400E070FA9000147401F022A0
:0100120022CB
:01006A002273
:010076002267
:108E84003038079000147402F02230370A20340777
:108E94009000147401F022303611900120E090000B
:108EA40006F0125361900006E070FA30370C90001F
:108EB400067405F0900006E070FA3036209000F554
:108EC400E0F53612B82CE4900170F01253FC9001D6
:108ED40070E004F0E0C3940A40F112B84B3037203C
:108EE4009000F6E0F53612B821E4900170F01253C8
:108EF400FC900170E004F0E0C3940A40F112B84B16
:108F040030360E90010CE0900001F0900001E0700A
:078F1400FAE4900014F022C2
:010077002266
:10B22F0030272C203929900013741EF0787EE6FF0A
:10B23F00547FFE900EFB93900015F0303C0DEF30D5
:10B24F00E709EE900F0B93900015F0D239C2272229
:10B25F0030252C203929900013741EF0787CE6FFDE
:10B26F00547FFE900EFB93900015F0303C0DEF30A5
:10B27F00E709EE900F0B93900015F0D239C22522FB
:105BEE00900274E0FF65797003025D89303903021B
:105BFE005D89900013741EF0EFD394FA4005E49083
:105C0E000274F0900274E0FF04F074752FF582E4D4
:105C1E003402F583E0FF647F7003025D89D239BFE1
:105C2E005D07900015745DF022BF5B079000157440
:105C3E005BF022BF30079000157430F022BF3107A1
:105C4E009000157431F022BF32079000157432F0B7
:105C5E0022BF33079000157433F022BF3407900033
:105C6E00157434F022BF35079000157435F022BF3D
:105C7E0036079000157436F022BF37079000157462
:105C8E0037F022BF38079000157438F022BF39075D
:105C9E009000157439F022BF23079000157423F07D
:105CAE0022BF2A07900015742AF022BF41079000E8
:105CBE00157441F022BF42079000157442F022BFC6
:105CCE0043079000157443F022BF640790001574CB
:105CDE0044F022203C03C23922BF610790001574A4
:105CEE0061F022BF62079000157462F022BF630755
:105CFE009000157463F022BF64079000157464F071
:105D0E0022BF65079000157465F022BF66079000EC
:105D1E00157466F022BF67079000157467F022BFF6
:105D2E0068079000157468F022BF6907900015741B
:105D3E0069F022BF6A07900015746AF022BF6B07E4
:105D4E00900015746BF022BF6C07900015746CF008
:105D5E0022BF6D07900015746DF022BF6E07900084
:105D6E0015746EF022BF6F07900015746FF022BF8E
:0B5D7E0070079000157470F022C2390D
:015D890022F7
:10002E00E4900170F0900170E0FFC39420501574BD
:10003E00172FF582E43400F5837420F0900170E000
:05004E0004F080E12236
:0FB7A600EFC394304007EFD39439500122C322F0
:10988700900020E0FD6420602E90001FE0540F75CB
:10989700F00AA4FBAAF090001EE0540F75F064A430
:1098A7002BFFE5F03AFEED540F7C002FFFEC3E90C6
:1098B70000D0F0A3EF803190001FE0FD64209000FE
:1098C7001E601AE0540F75F00AA4FFED540F7C00D8
:1098D7002FFEEC35F09000D0F0A3CE800BE0540FB4
:1098E700FF9000D0E4F0A3EFF0E024FFF09000D069
:0598F700E034FFF02247
:109E880090001DE0FD6420602B90001CE0540F75CD
:109E9800F00AA4FBAAF090001BE0540F75F064A42C
:109EA8002BFFE5F03AFEED540F7C002FFFEC3E90BF
:109EB80000D2802E90001CE0FD642090001B601AE8
:109EC800E0540F75F00AA4FFED540F7C002FFEEC50
:109ED80035F09000D2F0A3CEF022E0540FFF9000AE
:079EE800D2E4F0A3EFF02229
:10B5DA00900019E0540F75F00AA4FFA3E0540F2F4E
:10B5EA00900049F0D394004006E09415500122C31C
:01B5FA00222E
:1098FC00E4900170F0900170E0FFC394335064EF7A
:10990C0075F003A4241BF582E4340FF583E493FF74
:10991C0090001BE0FEEF6E7042900170E0FF75F05E
:10992C0003A4241CF582E4340FF583E493FE900029
:10993C001CE0FDEEB50524EF75F003A4241DF582A3
:10994C00E4340FF583E493FF90001DE0FEEFB506C1
:10995C000A900170E090004AF0D322900170E0046C
:05996C00F08092C3220F
:10979700E4900170F0900170E0FFC394705067751A
:1097A700F003EFA424B4F582E5F0340FF583E493D6
:1097B700FF90001BE0FEEF6E7044900170E0FF75B4
:1097C700F003A424B5F582E5F0340FF583E493FEA6
:1097D70090001CE0FDEEB5052575F003EFA424B657
:1097E700F582E5F0340FF583E493FF90001DE0FE6A
:1097F700EFB5060A900170E090004BF0D32290017C
:0898070070E004F0808FC32221
:107A470074172FF582E43400F583E0FE6431600398
:107A5700027ADB900170F0900170E0FDC39433501F
:107A67007074182FF582E43400F583E0FCED75F0AF
:107A770003A4241BF582E4340FF583E4936C704967
:107A870074192FF582E43400F583E0FD900170E06E
:107A9700FC75F003A4241CF582E4340FF583E4930A
:107AA700B50526741A2FF582E43400F583E0FDEC62
:107AB70075F003A4241DF582E4340FF583E493B530
:107AC7000507900170E004FF22900170E004F08048
:107AD700867F0022EE64326003027B68900170F0BB
:107AE700900170E0FEC39470507474182FF582E40F
:107AF7003400F583E0FD75F003EEA424B4F582E5C8
:107B0700F0340FF583E4936D704C74192FF582E40C
:107B17003400F583E0FE900170E0FD75F003A424C6
:107B2700B5F582E5F0340FF583E493B50628741AAA
:107B37002FF582E43400F583E0FE75F003EDA4240D
:107B4700B6F582E5F0340FF583E493B506089001A6
:107B570070E02434FF22900170E004F080827F00FF
:047B6700227F002257
:1094A900EFC394339000CB50397431F0EF75F0036A
:1094B900A4241BF582E4340FF583E4939000CCF0E7
:1094C900EF75F003A4241CF582E4340FF583E493CB
:1094D9009000CDF0EF75F003A4241DF582E4340F5C
:1094E900803A7432F075F003EFA4241BF582E5F09D
:1094F900340FF583E4939000CCF075F003EFA424C6
:109509001CF582E5F0340FF583E4939000CDF075F6
:10951900F003EFA4241DF582E5F0340FF583E493FD
:059529009000CEF022CD
:10B6B500900019E0540F75F00AA4FFA3E0540F2F72
:05B6C50090004CF02292
:10B6CA00900019E0540F75F00AA4FFA3E0540F2F5D
:05B6DA0090004DF0227C
:10B6DF00900019E0540F75F00AA4FFA3E0540F2F48
:05B6EF0090004EF02266
:10B4570090005EE0FF7E0090005FE0FCA3E0FD123D
:10B467007F0190005DE02FFF90005CE03EFE9000C2
:0AB4770055E07C002FFFEC3EFE22A2
:10B4FA00303608900037E0FF120086303708900097
:10B50A0037E0FF12005E30380D2059FD900037E019
:07B51A00900264F0D25922F7
:10A5A500E4900170F0900047E0FF900170E0FEC379
:10A5B5009F503F74372EF582E43400F583E0FF9019
:10A5C5000171E4F0A3EFF0303605E0FF12008630AC
:10A5D5003708900172E0FF12005E30380D2059FDFA
:10A5E500900172E0900264F0D259900170E004F09D
:03A5F50080B3220E
:10AC6100303838E4900170F0900170E0FFC3940433
:10AC7100502974CB2FF582E43400F583E0FF900175
:10AC810071E4F0A3EFF02059FD900172E0900264AD
:0CAC9100F0D259900170E004F080CD2258
:10AC9D00303838E4900170F0900170E0FFC39405F6
:10ACAD00502974CB2FF582E43400F583E0FF900139
:10ACBD0071E4F0A3EFF02059FD900172E090026471
:0CACCD00F0D259900170E004F080CD221C
:010078002265
:010079002264
:10AA690030383CE4900170F0900054E0FF900170A0
:10AA7900E0FEC39F502974372EF582E43400F58334
:10AA8900E0FF900171E4F0A3EFF02059FD9001720D
:10AA9900E0900264F0D259900170E004F080C9227C
:0C005E0012B6871253FC12B8520253FC79
:0C00860012B69E1253FC12B8520253FC3A
:1077F900E4900170F0900171F0A3F0900173F090A2
:1078090000D1E02401FD9000D0E03400FCC3ED94E8
:107819000AEC94005007A3E004900173F0D3ED94AF
:1078290063EC9400405D9000D1E02401FB9000D00E
:10783900E03400FA7C007D64AF03FE127F139001EF
:1078490070EFF0E075F064A4FFC3EB9FFFEA95F0D9
:10785900FE7C007D0A127F13900171EEF0A3EFF018
:107869009000D1E004FF900170E075F064A4FEC3BC
:10787900EF9EFF900172E075F00AA4FEC3EF9E909F
:107889000173F09000D1E02401FF9000D0E03400B2
:10789900FED3EF9409EE940040207C007D0A127F0C
:1078A90013900171EEF0A3EFF0E075F00AA4FF90D8
:1078B90000D1E004C39F900173F0900170E024307F
:1078C900F0900172E02430F0900171E03400F09002
:1078D9000173E02430F030361D900170E0FF120092
:1078E90086900172E0FF120086900173E0FF12009A
:1078F900867F2A12008630371D900170E0FF120042
:107909005E900172E0FF12005E900173E0FF1200C9
:077919005E7F2A12005E22CE
:06ABE6007BFF7A127908E2
:10ABEC008B188A19891A20382E7F01127D63E49004
:10ABFC000170F0900170E0FFC39410501AAB18AACA
:10AC0C0019A91A8F82758300127EC2FF127D3190B2
:08AC1C000170E004F080DC226D
:10A5F80090005CF0EFA3F090005E7403F0E490002C
:0AA608005FF0A3F07BFF7A1279588F
:10A612008B178A18891920382E7F11127D63E490D6
:10A622000170F0900170E0FFC39410501AAB17AAAA
:10A6320018A9198F82758300127EC2FF127D319094
:08A642000170E004F080DC224D
:10B481007BFF7A1279C812A612E4900170F0900144
:10B4910070E0FF7E00900E9793FD127592900170FF
:0AB4A100E004F0E0C3940240E5224D
:109399007BFF7A1279D812A612E4900173F0E49057
:1093A9000171F0A3F0E4900170F0900173E075F0A1
:1093B90099A42402FBE435F0FA900171E0FEA3E0E0
:1093C900FF7C007D03127F01EF2BFFEE3AFE900137
:1093D90070E0FD7A002FFFEA3EFEED900E9993FDB5
:1093E900127592900170E004F0E0C3940340BB90C1
:1093F9000172E004F07006900171E004F0C390017D
:1094090072E09433900171E094004099900173E007
:0994190004F0E0C3941440862223
:109167007BFF7A1279E812A612E4900173F0E4907B
:109177000171F0A3F0E4900170F0900173E0FF7EBD
:10918700007C017D50127F01EF24F6FBEE340BFAD1
:10919700900171E0FEA3E0FF1C7D03127F01EF2B1E
:1091A700FFEE3AFE900170E0FD7A002FFFEA3EFEE7
:1091B700ED900E9C93FD127592900170E004F0E023
:1091C700C3940340B5900172E004F07006900171FA
:1091D700E004F0C3900172E09470900171E0940094
:0F91E7004093900173E004F0E0C39414408022A1
:109BA3007BFF7A1279F812A612E4900174F0A3F005
:109BB300E4900170F0900170E0FBC39403502E9089
:109BC3000174E0FEA3E0FF7C007D03127F01EF241C
:109BD30036FFEE3426FEEB2FFFEC3EFEEB900E9F9E
:109BE30093FD127592900170E004F080C8900175A6
:109BF300E004F07006900174E004F0C3900175E096
:0B9C03009488900174E0941340A622A6
:01007A002263
:01007E00225F
:01007F00225E
:109C0E007BFF7A13793812A612E4900171F0A3F05B
:109C1E00E4900170F0900170E0FBC39456502E90CA
:109C2E000171E0FEA3E0FF7C007D56127F01EF2460
:109C3E00CEFFEE3460FEEB2FFFEC3EFEEB900EA55A
:109C4E0093FD127592900170E004F080C89001723D
:109C5E00E004F07006900171E004F0C3900172E030
:0B9C6E009414900171E0940040A622C5
:10B521007BFF7A13794812ABEC12B4811293991212
:10B531009167129BA312007A12007E12007F129C67
:07B541000E127D80027D92D5
:10B4AB00E49000D4F0A3F0FFFE1275D39000A8EF48
:10B4BB00F09000D5E02401FF9000D4E03400FE12A0
:08B4CB0075D39000D6EFF022CA
:108ABC00756D01756E00756FE9E4900378F0A3F0A5
:108ACC00900378E0FAA3E0FBC39456EA940050407C
:108ADC009000A8E075F056A42478FFE5F03460CF40
:108AEC002BCF3AFE9000D4F0A3EFF01275D3AB6D00
:108AFC00056FE56FAA6E7002056E14F9EF127EEF2A
:108B0C00900379E004F070B8900378E004F080B042
:108B1C00900116E024FF924B900115E024FF923255
:108B2C00900135E0F537900136E0F53890011CE006
:108B3C0024FF924A90011BE024FF923390011AE02B
:108B4C007004D2558002C255900113E024FF922389
:0A8B5C009000A974FFF09000AAF049
:018B660022EC
:10A13100756D01756E01756F48E4900378F0A3F0B9
:10A14100900378E0FEA3E0FFC39414EE9400503B2B
:10A151007C007D56127F01EF24F9FFEE3460FE9002
:10A1610000D4F0A3EFF01275D3AB6D056FE56FAAC4
:10A171006E7002056E14F9EF127EEF900379E00420
:0BA18100F070BD900378E004F080B5A2
:01A18C0022B0
:10A18D00756D01756E01756F5CE4900378F0A3F049
:10A19D00900378E0FEA3E0FFC39414EE9400503BCF
:10A1AD007C007D56127F01EF24FEFFEE3460FE90A1
:10A1BD0000D4F0A3EFF01275D3AB6D056FE56FAA68
:10A1CD006E7002056E14F9EF127EEF900379E004C4
:0BA1DD00F070BD900378E004F080B546
:01A1E8002254
:1091F6008F17E4900170F0900170E0FBC394035068
:109206003E9000A8E075F099A42469FDE5F034FFCE
:10921600FCE51775F003A42DFFE5F03CFEEB7C00A2
:109226002FFFEC3EFE1275D3900170E024DEF5822E
:10923600E43400F583EFF0900170E004F080B8901C
:1092460000DEE0FE54019000D7F0EE54029000D804
:10925600F09000DEE054049000D9F0EE540890003F
:10926600DAF09000DEE054109000DBF09000DFE0D2
:0D9276009000DCF09000E0E09000DDF022C0
:109043008F17E4900170F0900170E0FBC39403501C
:10905300449000A8E0FF7E007C017D50127F01EF69
:1090630024A6FDEE340AFCE51775F003A42DFFE5F5
:10907300F03CFEEB7C002FFFEC3EFE1275D390011B
:1090830070E024DEF582E43400F583EFF0900170A4
:10909300E004F080B29000DEE0FE54019000D7F0CF
:1090A300EE54029000D8F09000DEE054049000D912
:1090B300F0EE54089000DAF09000DEE054109000D7
:1090C300DBF09000DFE09000DCF09000E0E0900047
:0390D300DDF022AB
:068C0D008F178C188D1971
:108C1300E4900378F0A3F0E51924FFFFE51834FF8F
:108C2300FE7C007D03127F01AA06AB07AE17E51792
:108C330025E0CE75F0EEA4FFE5F02EFEEF2448FF0D
:108C4300EE3423CF2BCF3AFE900379E02FFF90032E
:108C530078E03EFE1275D3900379E024DEF582E4DA
:108C63003400F583EFF0900379E004F0700690038D
:108C730078E004F0C3900379E09403900378E094E0
:108C83000040949000DEE0FE54019000E4F0EE54C6
:108C9300029000E5F09000DEE054049000E6F090CE
:0F8CA30000DFE09000E7F09000E0E09000E8F0E4
:018CB200229F
:103D28007BFF7A0079A612ABEC12AE3DE490025FFD
:103D3800F0A3F090017304F0900173E0C394154070
:103D480003023EFF900174E4F0A304F0C3900175F0
:103D5800E094FB900174E094004003023EF6900169
:103D680073E0FF7E007C027DEE127F01EF2448FFA6
:103D7800EE342390005CF0FAA3EFF0FB900175E0BD
:103D880024FFFF900174E034FFFE7C007D03127F66
:103D980001EF2BFFEE3AFE1275D3EF54029000DECE
:103DA800F0900175E024FFFF900174E034FFFE7C81
:103DB800007D03127F0190005DE02FFF90005CE022
:103DC8003EFE1275D3EF54049000E1F09000DEE05F
:103DD8007003023EE29000E1E07003023EE29001CF
:103DE80074E0FEA3E0FF7C007D03127F0190005D7C
:103DF800E02FFF90005CE03ECF24FECF34FFFE12A0
:103E080075D39000DFEFF0900174E0FEA3E0FF7C33
:103E1800007D03127F0190005DE02FFF90005CE0C1
:103E28003ECF24FFCF34FFFE1275D39000E0EFF0B1
:103E3800FD9000DFE0FF12553B900171EEF0A3EF1B
:103E4800F04E7003023EE290025FE475F001127FCB
:103E580068AFF0FE900173E0FD12A77990025FE46D
:103E680075F001127F68AFF0FE900175E0FD12A7B2
:103E78007990025FE475F001127F68AFF0FE900060
:103E8800DFE0FD12A77990025FE475F001127F6808
:103E9800AFF0FE9000E0E0FD12A779D3900260E059
:103EA800948890025FE0941340307BFF7A0079B7E2
:103EB80012ABEC90025FE0FEA3E07802CEC313CE13
:103EC80013D8F9F0EE90025FF09000057414F090AA
:103ED8000005E070030241B080F5900175E004F040
:103EE8006003023D54900174E004F0023D549001D7
:103EF80073E004F0023D40E4900170F0900170E03E
:103F0800FBC3943340030240379000A8E075F09952
:103F1800A42469FDE5F034FFFCEB75F003A42DFF44
:103F2800E5F03CFE90005CF0A3EFF01275D3900032
:103F3800DEEFF054049000E1F09000DEE0541090C1
:103F480000E2F09000E1E0700302402EA3E070036D
:103F580002402E90005DE02401FF90005CE03400F8
:103F6800FE1275D39000DFEFF090005DE02402FFB1
:103F780090005CE03400FE1275D39000E0EFF0FD95
:103F88009000DFE0FF12553B900171EEF0A3EFF0D7
:103F98004E700302402E90025FE475F001127F68B4
:103FA800AFF0FE7D1512A77990025FE475F001125B
:103FB8007F68AFF0FE900170E0FD12A77990025F74
:103FC800E475F001127F68AFF0FE9000DFE0FD12AB
:103FD800A77990025FE475F001127F68AFF0FE9058
:103FE80000E0E0FD12A779D3900260E09488900287
:103FF8005FE0941340307BFF7A0079B712ABEC9006
:10400800025FE0FEA3E07802CEC313CE13D8F9F026
:10401800EE90025FF09000057414F0900005E070D7
:10402800030241B080F5900170E004F0023F04E41F
:10403800900170F0900170E0FBC39470400302415E
:10404800919000A8E0FE75F050A4FFE5F02EFEEF79
:1040580024A6FDEE340AFCEB75F003A42DFFE5F071
:104068003CFE90005CF0A3EFF01275D3EF5404907F
:1040780000DEF090005CE0FEA3E0FF1275D3EF5481
:10408800109000E1F09000DEE0700302418890009B
:10409800E1E0700302418890005DE02401FF900098
:1040A8005CE03400FE1275D39000DFEFF090005D05
:1040B800E02402FF90005CE03400FE1275D390000B
:1040C800E0EFF0FD9000DFE0FF12553B900171EE4C
:1040D800F0A3EFF09000DEE070030241889000E169
:1040E800E07003024188900171E07002A3E0700360
:1040F80002418890025FE475F001127F68AFF0FE1C
:104108007D1612A77990025FE475F001127F68AFFF
:10411800F0FE900170E0FD12A77990025FE475F05F
:1041280001127F68AFF0FE9000DFE0FD12A77990E2
:10413800025FE475F001127F68AFF0FE9000E0E0E6
:10414800FD12A779D3900260E0948890025FE09412
:1041580013402D7BFF7A0079B712ABEC90025FE039
:10416800FEA3E07802CEC313CE13D8F9F0EE900286
:104178005FF09000057414F0900005E0602A80F864
:10418800900170E004F002403C90025FE0FEA3E082
:104198007802CEC313CE13D8F9F0EE90025FF07B0D
:0941A800FF7A0079C812ABEC2289
:10A69900AB07AA067C007D64127F13EF443090005B
:10A6A900CBF07C007D64AF03AE02127F137E007F86
:10A6B9000ACFCDCFCECCCE127F13EF4430A3F0AE6C
:10A6C90002AF037C007D64127F137E007F0ACFCD29
:0DA6D900CFCECCCE127F13ED4430A3F02283
:10B1FD00900022E0540F75F00AA4FDACF0900021F0
:10B20D00E0540F75F064A42DFFE5F03CFE90002393
:10B21D00E0540F7C002FFFEC3EFE900171F0A3EF88
:02B22D00F0220D
:10A551002A2A3132333435362A2A2A2A31323334FF
:10A5610035302A2A44313233343536373839302AB6
:10A571002341424320464C45582049562020412042
:10A58100322E30302020202020534C4156452020AF
:10A591002020202020202020204D415354455220AE
:04A5A1002020202036
:1088A900303F23C23F787EE6540F90A5659390012F
:1088B9008AF09000077432F09000EAE0601612AD79
:1088C900C712A809800E900007E07008900176F0A1
:1088D900900187F0304049C240787CE6540F90A55A
:1088E9006593900189F09000087432F090025EE07F
:1088F900FF60069000E9E07009EF70099000EBE075
:10890900600312A7C290025EE0FF60069000E9E0F2
:108919007003EF700312AD8C20341312B197800EDF
:10892900900008E07008900177F0900186F09002BD
:1089390074E0FF657960149000ECE06018EFD3945F
:10894900FA4005E4900274F0027FA4900009E070F7
:0689590004900273F022FD
:10AD8C00900177E0FF04F0EF90A55193FF900189BB
:10AD9C00E0FEEF6E6011EEB42A089001777401F0BA
:10ADAC008005E4900177F0900177E0B40A0C12531F
:0BADBC0067E4900177F0D237D241220B
:10ADC700900176E0FF04F0EF90A55193FF90018A80
:10ADD700E0FEEF6E6011EEB42A089001767401F080
:10ADE7008005E4900176F0900176E0B40A0C1253E6
:0BADF70067E4900176F0D236D24122D2
:10A7C200900186E0FF04F0747D2FF582E43401F5F8
:10A7D20083E0FF900189E0FEEF6E6011EEB4230882
:10A7E2009001867401F08005E4900186F090018664
:10A7F200E0B40912125373125367120056E4900127
:07A8020086F0D237D23522A7
:10A80900900187E0FF04F0747D2FF582E43401F5AF
:10A8190083E0FF90018AE0FEEF6E6011EEB4230839
:10A829009001877401F08005E4900187F090018719
:10A83900E0B40912125373125367120056E49001DF
:07A8490087F0D236D2352260
:10B19700900179E0FF04F0EF90A55B93FF900189A0
:10B1A700E0FEEF6E6011EEB42A089001797401F0A9
:10B1B7008005E4900179F0900179E0B40A04E4F0A5
:03B1C700D242224F
:10B3A50090017D7423F0A3F0E4FF74ED2FF582E4A2
:10B3B5003400F583E0FE747F2FF582E43401F583D4
:0CB3C500EEF00FBF06E49001857423F049
:01B3D1002259
:109FB900127C8E127D80127D927F01127D637BFF60
:109FC9007AA5797512ABEC90011AE07BFF60067AED
:109FD900A5798580047AA5799512A6129000057451
:109FE9001EF0E490017BF090017CF0FF74AB2FF53B
:109FF90082E43400F583E4F074BB2FF582E4340085
:10A00900F583E4F00FBF10E4900005E070FA027DDB
:01A0190080C6
:1096A40090017BE0FFD3940F501FEF04FF127D6302
:1096B400900189E0FF90017BE0FE04F074AB2EF58D
:1096C40082E43400F583EF804C7F01127D63E490E3
:1096D4000170F0900170E0FFC3940F5030E0FE245D
:1096E400ACF582E43400F583E0FD74AB2EF582E43E
:1096F4003400F583EDF074AB2FF582E43400F58388
:10970400E0FF127D31900170E004F080C690018981
:0A971400E0FF9000BAF0127D312250
:1095AE0090017CE0FFD3940F5020EF2411FF127D29
:1095BE006390018AE0FF90017CE0FE04F074BB2E04
:1095CE00F582E43400F583EF804C7F11127D63E465
:1095DE00900170F0900170E0FFC3940F5030E0FEE8
:1095EE0024BCF582E43400F583E0FD74BB2EF582D5
:1095FE00E43400F583EDF074BB2FF582E43400F50E
:10960E0083E0FF127D31900170E004F080C690017E
:0B961E008AE0FF9000CAF0127D3122AC
:107FA400900273E0FF702C900274E0FE04F074758C
:107FB4002EF582E43402F583E090017AF090000912
:107FC4007432F090017AE0FEB41B02D241EEB47E2A
:107FD400028064EFB4012A900274E0FF04F0747527
:107FE4002FF582E43402F583E090017AF0900009E1
:107FF4007432F090017AE0B45002803BE490027352
:10800400F0900273E06402703A900274E0FF04F0AE
:1080140074752FF582E43402F583E090017AF090D0
:1080240000097432F09000D6E075F00A844430FF01
:1080340090017AE0B50707900273E004F022E4901F
:108044000273F0900273E064037044900274E0FFE2
:1080540004F074752FF582E43402F583E090017A1C
:10806400F09000097432F0E4900273F09000D6E0CE
:1080740075F00A84E5F04430FF90017AE0B5070F0B
:10808400E4900014F0D238D235D239C250C2512211
:105D8A00755900125DA550FB22755900125E2E50FE
:105D9A00FB22755900125DE550FB22758400E55916
:105DAA0075F003A4905DB273025E4A025E59025E08
:105DBA0077025E60025E83025E8A025E92025E592A
:105DCA00025EA0025E60025EB0025EB9025E4A0234
:105DDA005E59025EC7025E60025ED3758400E559B1
:105DEA0075F003A4905DF273025E4A025E59025E88
:105DFA0077025E60025E83025E8A025E4A025E5932
:105E0A00025E77025E60025E83025E8A025E83023F
:105E1A005E8A025E92025E59025ED5025E60025E90
:105E2A00B0025ED3758400E55975F003A4905E3B19
:105E3A0073025E4A025E59025EC7025E60025ED368
:105E4A00C2FA125EE5125EE5759B000559C322305F
:105E5A00F9020559C32230F912E59A20E7FB125ECE
:105E6A00E5D2FA125EE5125EE50559C322C2FA12BC
:105E7A005EE5759B040559C32275411E0559C32267
:105E8A00E54170020559C322C2FA125EE5125F06A5
:105E9A00F59B0559C322C2FA125EE5125F15440743
:105EAA00F59B0559C322125EF7F5420559C32275BF
:105EBA00840F30DE04E54270020559C322C2FA1289
:105ECA005EE5759B080559C322D322C2FA125EE524
:095EDA00125F154405F59B055902
:105EE300C3220000000000000000000000000000CA
:105EF30000000022905EFEE55A93225A5A5A5A5ADB
:105F0300FAFAFA905F0DE55A932200B45AE12D870D
:105F13007ADB905F1CE55A932200000000000080AA
:015F230080FD
:1013E800C0D0C000C001C083C082C0E0C0F0C00748
:1013F800A292304B01B3787BE233F208E233F20871
:10140800E233F208E233F208E233F208E233F20898
:10141800E233F208E233F208E233F208E233F20888
:10142800E233F208E233F208E233F208E233F20878
:10143800E233F208E233F208E233F208E233F20868
:10144800E233F208E233F208E233F208E233F20858
:10145800E233F208E233F208E233F208E233F20848
:10146800E233F208E233F208E233F208E233F20838
:10147800E233F208E233F208E233F208E233F20828
:01148800E281
:1014890033F208E233F208E233F208E233F208E217
:1014990033F208E233F2305C359018B478A2E218DE
:1014A900202303936028E218937023E21893601EA7
:1014B900E218937019E218936014E21893600FE22E
:1014C9001893700AE218937005E2189360030216E4
:1014D9008E755000E2189313924350037550387576
:1014E9002300E2189313921C500363501CE21893D3
:1014F90013921B500363500EE2189313921A500370
:10150900635046E218931392195003635023E2186B
:10151900931392188523515003635051752300E2A8
:10152900189313921C5003635068E2189313921B8B
:101539005003635075E2189313921A500363507A5B
:10154900E21893139219500363503DE218931392D2
:1015590018852352500363501F752300E218931313
:10156900921F500363504FE2189313921E50036366
:101579005026E2189313921D5003635052E21893B8
:1015890013921C5003635029E2189313921B5003C2
:10159900635015E2189313921A500363500BE21823
:1015A900931392195003635045E2189313921885C7
:1015B90023535003635062E2189313921C50036340
:1015C9005031E2189313921B5003635019E2189398
:1015D90013921A500363500DE21893139219500392
:1015E900635007E2189313921885235450036350EC
:1015F90043752300E2189313921EE2189313921D68
:10160900E2189313921CE2189313921BE218931396
:10161900921AE21893139219E218931392188523D8
:1016290055C248E55565506035D24823F8901E05E6
:1016390093F9901E04E8936025B40104B243801E17
:0E164900B40205E862518016B40305E862524F
:10165700800EB40405E862538006B4052AE8625494
:10166700A24392449000A3E551F09000A4E552F004
:101677009000A5E553F09000A6E554F0304706D258
:1016870046C2478002D2471216A2D007D0F0D0E058
:10169700D082D083D001D000D0D022C0D0C000C02B
:1016A700E0302D4EE562B40833A230B392B37880B0
:1016B700E66036167885E6A2E7303201B3923092BB
:1016C700B2A2E77881E633F67882E633F67883E6E6
:1016D70033F67884E633F67885E633F6D562037514
:1016E7006208D0E0D000D0D022C254D0E0D000D0E1
:1016F700D022D0E0D000D0D022C0D0C000C001C0DE
:1017070083C082C0E0C0F0A292204A01B37863E2AE
:1017170013F208E213F208E213F208E213F208E206
:1017270013F208E213F208E213F208E213F208E2F6
:0D17370013F208E213F208E213F208E213C5
:10174400F208E213F208E213F208E213F208E213D9
:10175400F208E213F208E213F208E213F208E213C9
:10176400F208E213F208E213F208E213F29018B45A
:101774007863E20893139217E20893139216E2082F
:1017840093139215E20893139214E208931392139D
:10179400E20893139212E20893139211E20893134E
:1017A4009210852256E20893139217E2089313923B
:1017B40016E20893139215E20893139214E2089325
:1017C400139213E20893139212E20893139211E214
:1017D4000893139210852257E20893139217E20894
:1017E40093139216E20893139215E208931392143A
:0117F400E212
:1017F5000893139213E20893139212E2089313923B
:1018050011C210852258305C3DE556901C04855761
:1018150022301602058393602D14F875F003A49009
:101825001AB52582F582E5F03583F583E493F9A3AE
:10183500E4939019B4655893C965579329B4010089
:1018450050048844D22F12185DD0F0D0E0D082D059
:1018550083D001D000D0D022302B26788616E670B2
:101865002076087889E6A2E1303301B392B292B3CB
:10187500A2E17887E613F67888E613F67889E61309
:10188500F622EF901AB475F003A42582F582E5835C
:1018950035F0F583C22B7400937887F6740193783D
:1018A50088F67402937889F6C22DC22CD22B2200B9
:1018B5000000000000000000000000000000000023
:1018C5000000000000000000000000000000010012
:1018D5000000000000000000000000000000010002
:1018E50000000000000001000000010001010100EE
:1018F50000000000000000000000000000000100E2
:1019050000000000000001000000010001010100CD
:1019150000000000000001000000010001010100BD
:1019250000000100010101000101010101010100A7
:1019350000000000000000000000000000000100A1
:10194500000000000000010000000100010101008D
:10195500000000000000010000000100010101007D
:101965000000010001010100010101010101010067
:10197500000000000000010000000100010101005D
:101985000000010001010100010101010101010047
:101995000000010001010100010101010101010037
:1019A5000101010101010101010101010101010023
:1019B5000101020102020301020203020303040101
:1019C50002020302030304020303030303040501E4
:1019D50002020302030304020303040304040502D1
:1019E50003030403040405030404040405050601B4
:1019F50002020302030304020303030304040502B2
:101A05000303040303040503040405040505060292
:101A15000303040304040503040405040505060380
:101A25000404050405050604050506050606070163
:101A35000202030203030402030304030404050270
:101A45000303040304040503040405040505060251
:101A55000303040304040503040405040505060340
:101A65000404050405050604050506050606070222
:101A75000303040304040503040405040505060320
:101A85000404050405050604050506050606070301
:101A950004040504050506040505060506060704F0
:101AA500050506050606070506060706070708FDD8
:101AB500D00C73700E3CF01AAF101E7F9022EC70A4
:101AC50026D6F02ACBB02CA3F032BEB03417D03CCA
:101AD500B6D0461FB04E77F050F950526AB056DE78
:101AE5009058BA306ACF3072D270745CD076E8F014
:101AF500786BD098E5709AF8309CBB50A40F70AA0B
:101B05007A70B26730B45DB0B8FCB0C26F50C655DC
:101B1500D0CA3D90D489B0DA94F0DCD790E463B0B4
:101B2500EA0BF0F43170F8DD310AB571148FF11854
:101B3500D1D126EB512AF6112C8B71463F5148B174
:101B4500F14AACB14CC4F152D9B1546D915A2EF150
:101B550062BD116687916A9AD16CF29172D55178FE
:0D1B650019F18C71B192D8D19A32D1AA47F2
:101B7200D1B25A91B452F1C67531CC1D71D2A9516C
:101B8200DCD0B1E85E11EA2B11F2EED212F392141C
:101B92007D3216973226D8B232C5F234F7124AEAAB
:101BA200524C9F5254A5D2582B725A7552644FD23E
:101BB20068C1726ADC326C78D2865F128C83729C46
:101BC2004EB2A66972AC1C72B433D2CC18F2EABB24
:101BD200330CCE33141EB32803F32EE51332F8531D
:101BE2003498735848F36472736845738617B394D4
:101BF2007313A63C93B221D3B41B53B829B3C64185
:101C0200F3D8000000000000000000000000000007
:101C12000000000000000000006A00000000000058
:101C2200620D0000000000000000006F004800008C
:101C320000000000000000000000000000006C2214
:101C42000000000000000000000000000000000092
:101C52005B00000000000000000000004100001EC8
:101C62004759000000260000001D0000100000354A
:101C72000000003D006B0043000000000000004B2C
:101C820000050000000000000038002300000000F2
:101C92000000000000000000004C000000000000F6
:101CA2000000000000000000000000000000320000
:101CB2000004000000000000000000001260003775
:101CC2000A00000000000000000000000008000000
:101CD200611346000000000000254D340000572922
:101CE200110000000000006400000000000000007D
:101CF200000000003A4A00002E4F190000001F00A9
:101D02000000000000630000000000000027000047
:101D1200001B000000000000000B5F3C006E5D44F1
:101D22000000006D000000000000000000530000F1
:101D3200360000283F5E00000000000000000300A3
:101D420000300070000000690040670000000000E1
:101D520000550000420000210000000000001500B4
:101D620000000000000000000000005C00170000FE
:101D72000020000068020054000E58001C00000001
:101D820000000000005A000000000000002F0000C8
:101D9200002B000000002400000066003900000053
:101DA2000051000000090052000000450000000040
:101DB200000000310000002A0C000000001A0000A0
:101DC200000000560000334E00000000000000003A
:101DD2000000002C1400003B07003E000000000041
:101DE200000000000000001800001600502D060040
:101DF20049000000000000000000650F0000000123
:101E020000000000000000000600000006000600BE
:101E12000502060006000600040406000504020886
:101E22000600000006000600060006000408060080
:101E3200060006000508060006000210060006005D
:101E4200030100000600060002020600060004402C
:101E52000600060004100600060006000600060042
:101E62000600060005100600060006000600060031
:101E72000600010106000600060006000302060035
:101E82000600000006000600050106000402020426
:101E92000600060006000600060006000600060010
:101EA2000480060002010420060006000600060067
:101EB20006000600060006000600060006000600F0
:101EC20006000600060004010600060006000600E1
:101ED20006000310060006000600060006000600C3
:0D1EE20006000600060006000600060003CC
:101EEF0008060006000600060003040600060006AA
:051EFF000006000600D2
:1048D700758400C2CA85CC4885CD4775CC0075CD97
:1048E70000D2CA10CF02D25B32305B0BC25BE54706
:1048F700C3943640028001227891798F7B06E7F6D0
:104907001819DBFAA64718A648AA48AB47AE02AF64
:1049170003EEC4035407FEEFC403FF54F84EFEEF43
:104927005407FF7803798CC3E79AFC09E79BFD09D5
:1049370050066304FF6305FFC3EC9EED9F5074D8D8
:10494700E6789979977C06E7F61819DCFAA6031832
:10495700A6027994AE02AF03EEC423541FFEEFC440
:1049670023FF54E04EFEEF541FFF7803C3E79AFC82
:1049770009E79BFD0950066304FF6305FFC3EC9E2F
:10498700ED9F502FD8E678927A007B007C0079045F
:10499700EA26FA08EB36FB08EC3400FCD9F2EC13F4
:0D49A700FCEB13FBEA13FAEC13EB13F546DF
:1049B400EA13F545D22122302131C2211249F050A7
:1049C4002A854C4D854B4C854A4B85494A85074978
:1049D400302013E54F6F600EE507B54A0EB54B0B5B
:1049E400B54C08B54D0585074ED22222904B0BE5F8
:1049F4004693FF904A3723232582F582E5833400CA
:104A0400F583124A16400A0F124A1640040F124A3E
:104A14001622E493F9A3E493FAA3E493FBA3E493A7
:104A2400FCA3C3E5459AE546995007C3EC9545EBCD
:104A3400954622EA25DD89DD89D324D324CBD2CB44
:104A4400D2C4DBC4DBBE39BE39B7CAB7CAB18EB172
:104A54008EAB87AB87A59CA59CA000A0009A969AD4
:104A64009695D895D891E591E58D858D8588AF8803
:104A7400AF840C840C7F9A7F9A7B497B49771B77A0
:104A84001B730F730F6F276F276B576B5767AB67DA
:104A9400AB642C642C60C660C65D795D795AFE5A9D
:104AA400FE5970597057E257E25661566154E75403
:104AB400E7537453745207520750A050A04F404F0D
:104AC400404DE64DE64C934C934B414B4149F549DF
:104AD400F548B548B547764776463E463E450845CF
:104AE40008432A432A40E440E43F533F533E3E3EBA
:104AF4003E3C943C943A863A863918391838050075
:104B040000000000000000323232323232323232DF
:104B14003232323232323232323232323232323271
:104B24003232323232323232323232323232323261
:104B34003232323232323232323232323232323251
:104B4400313130302F2E2D2D2D2C2C2B2A29292894
:104B540027262525242323222120201F1E1E1D1C39
:104B64001C1B1A1A1A1A19191918181817171717B3
:104B740016161616151515151414141413131313E9
:104B8400121212121111111110101010100F0F0F18
:104B94000F0F0E0E0E0E0D0D0D0D0C0C0C0C0B0B41
:104BA4000B0B0B0B0A0A0A0A0A0909090909090865
:104BB4000808080808070707070707060606060681
:104BC4000606050505050505040404040404040398
:104BD40003030303030302020202020202010101AE
:104BE40001010101010101010101010000000000B6
:104BF40000000000000000000000000000000000B1
:104C040000000000000000302C0D852F8A852E8CBA
:0A4C1400D28CB2B1D2A932C28C22B8
:10706300C007C0007F01127D637F4C127D317F54C6
:10707300127D317F52127D317F20127D31204404F5
:107083007F3080027F31127D317F20127D3190006D
:10709300A4E0785D1254CF785D8607430730127DF4
:1070A30031088607430730127D31750720127D3181
:1070B3009000A5E0785D1254C7785D8607430730DA
:1070C300127D31088607430730127D310886074356
:1070D3000730127D31750720127D319000A3E078CF
:1070E3005D1254CF785D8607430730127D310886E1
:1070F30007430730127D31750720127D31D000D050
:107103000722C007C0007F11127D637F4C127D31BF
:10711300750720127D312049047F3080027F3112B0
:107123007D317F20127D319001F9E0785D1254CFDB
:10713300785D8607430730127D31088607430730A1
:10714300127D31750720127D319001FAE0785D12CE
:1071530054C7785D8607430730127D31088607439D
:107163000730127D31088607430730127D317507DA
:1071730020127D319001FBE0785D1254CF785D865B
:1071830007430730127D31088607430730127D31EC
:10719300750720127D319001FCE0785D1254CF78A1
:1071A3005D8607430730127D310886074307301297
:0771B3007D31D000D007225E
:106AEE00003800512372461765340E5F2D7C48190D
:106AFE006B3A1C4D3F6E5A0B792812433160540588
:106B0E007726001F3D227A654758756A48570F1041
:106B1E00322D6877554A120D2F301D02203F6778AF
:106B2E005A45006245270B694E2C157750321E7C54
:106B3E005B39294B6C0E224067053C5E791B37553D
:106B4E00721052301775593B1C7E472502604C2E31
:106B5E00096B7B193E5C701235576E0C2B4965071D
:106B6E002042264463012D4F680A33517614385A59
:106B7E007D1F0F6D4A28046641231A785F3D1173FD
:106B8E005436741631537F1D3A58610324466A08F1
:106B9E002F4D5D3F187A56341371482A0D6F4321DD
:106BAE0006644F2D0A68442601635A381F7D5133FF
:106BBE001476660423416D0F284A73113654781AE1
:106BCE003D5F1D7F583A16745331086A4D2F03618D
:106BDE004624345671133F5D7A18214364062A48C1
:106BEE006F0D690B2C4E620027457C1E395B7715A5
:106BFE003250402205674B290E6C553710725E3CA1
:106C0E001B793B597E1C305275172E4C6B0925474C
:106C1E00600212705735197B5C3E076542200C6E80
:106C2E00492B004307440D4E0A49195A1E5D14574D
:106C3E001350317236753C7F3B78286B2F6C25666E
:026C4E002261C1
:108D5000788576ACA249E433FFC4333354C0FE9027
:108D600001FBE0FD541F25E04EFE9001F9E0FC54AC
:108D700010C4540F4E7884F6EC540FC454F0FE9097
:108D800001FAE0FC54F0C4540F4E7883F6EC540F13
:108D9000C454F0FE9001FCE0FC541EC3134E7882D4
:108DA000F6EF3395E0FE74EE2FF582746A3EF5839C
:108DB000E493FFED906AF093FEEF6EFF9001F9E00F
:108DC000906B10936FFF9001FAE0906B30936FFF00
:108DD000EC906C30936F7881F69001FCE030E00409
:0B8DE000E64480F6D25478807628220A
:10A4FC00758401309914C299204C0F9001F7E070CB
:10A50C0009D24CD29C789A7604223098379001F874
:10A51C00E06401702DE55B75F00584205211248DEB
:10A52C00F582E43401F583E599F0C298D2522224E5
:10A53C00A2F582E43401F583E599F0C298C252D2B7
:05A54C005322C2982219
:10832A007584012098030283F0204E13209A0DE5EC
:10833A00997009D24ED24F755C0AF55BC2982290A9
:10834A0001F8E0FF6401702CE55B75F005842052AA
:10835A0010248DF582E43401F583E599F0D2528038
:10836A001024A2F582E43401F583E599F0C252D2D1
:10837A0053C29822EFB4021AAB6D056FE56FAA6E6D
:10838A007002056E14F9E599127EEF9001F87403F4
:10839A0080209001F8E0FFB4031CAB6D056FE56F18
:1083AA00AA6E7002056E14F9E599127EEF9001F833
:1083BA007404F0C29822EFB4042990022AE0FF0460
:1083CA00F074012FF582E43402F583E599F0C2983E
:1083DA0090022AE0B4281C90022C7401F0E4900167
:1083EA00F8F022C2982230990AC2999001F7E070F7
:0483FA0002C2522247
:10B54800204D2212538C43E740755C0AE4F55B906A
:10B5580001F7F09001F8F0C24CD24D75840175984E
:06B5680090C29CF599223F
:109F560090022BE0705C90036FE0FF7025D39001B8
:109F6600FEE094869001FDE094674008E4F0A37457
:109F760002F0800E9001FEE02428F09001FDE0340E
:109F860000F09001FEE02FFF9001FDE03400FE128C
:109F960075D390036FE02401F582E43402F583EF74
:109FA600F090036FE004F0E0B42807E4F090022B91
:039FB60004F02292
:1090D60090022CE070030291669001FFE0FEA3E08F
:1090E600FFC39402EE94005006E490022CF0229006
:1090F600036FE07C002FFFEC3EFE1275D390036FEA
:10910600E02401F582E43402F583E0FD6F601790F8
:10911600036FE0FF900200E02FFF9001FFE03400B4
:10912600FE127592D25090036FE004F0E06428704E
:109136002F90022CF090036FF09001FFE0FEA3E069
:10914600FFBE2008BFD205E490036FF0EF64024E25
:10915600700E30500BC250128ABC12A13112A18D72
:0191660022E6
:109E2000304C6475840190023EE0B40D00505590B2
:109E30009E36F8282873029E5D029E60029E630291
:109E40009E66029E69029E6C029E6F029E72029E38
:109E500075029E78029E7B029E7E029E8102B3491D
:109E600002B6F402A91D02ACD902B5B702001E0267
:109E7000B1CA02AFFD02AD1502A96002B65502B328
:089E8000FF02B63A12B66F2290
:10B34900789AE67028759898755C0AF55B9000A85C
:10B35900E0B4010790023E7404F022E49001F8F091
:0EB369009001F7F090023EE004F012538922AA
:10B6F4009001F87401F0E49001F7F0C25290023E18
:04B70400E004F0224B
:10A91D009000A8E01475F005A4B55B19E4B5F01529
:10A92D0075989812538CE49001F7F09001F8F0901F
:10A93D00023E7404F0E55B75F00584AFF0BF0112C3
:10A94D00C253E49001F7F09001F804F090023EE05C
:03A95D0004F022E1
:10ACD900E55B75F00584AFF0BF043020531EE55BDA
:10ACE90075F00584FF248DF582E43401F583E4F0E1
:10ACF90074A22FF582E43401F583E4F0E49001F7BE
:0CAD0900F09001F8F090023EE014F022FF
:10B5B7009000A8E075F005A424FDB55B159000A9DF
:10B5C700E0F599E49001F7F09001F8F090023EE081
:03B5D70004F0225B
:0D001E009000AAE0F59990023EE004F02267
:10B1CA009000A8E0FD75F005A4FFE55BB50723E450
:10B1DA00B5F01FEDB4140790023E7409F022125321
:10B1EA0089E49001F7F0C2529001F8F090023EE033
:03B1FA0004F0223C
:10AFFD00E55BB4641212538CE49001F7F09001F804
:10B00D00F090023E7409F0E55B75F00584AFF0BF7A
:10B01D000112C253E49001F7F09001F804F0900290
:05B02D003EE004F022EA
:10AD1500E55B75F00584AFF0BF043020531EE55B9D
:10AD250075F00584FF248DF582E43401F583E4F0A4
:10AD350074A22FF582E43401F583E4F0E49001F781
:0CAD4500F09001F8F090023EE014F022C3
:10A96000E55B6465703C90022BE0B4012F756D01CE
:10A97000756E01756FFDE49001F7F09001F8F075C8
:10A980008401AB6D056FE56FAA6E7002056E14F958
:10A99000127EA9F59990023EE004F02290023E74E6
:03A9A0000CF02296
:10B65500758401AB6DAA6EA96F127EA9F599E49068
:0AB665000229F090023EE004F022FA
:10B3FF00758401900229E0FF04F074012FF582E4B7
:10B40F003402F583E0F599900229E0D39428400B9C
:0CB41F00E490022BF090023EE004F022CA
:10B63A00E55BB46915C24CC24DE490018BF09001F0
:0BB64A00F7F09001F8F090023EF022B3
:10B66F00C24CC24DE4F55B90018BF09001F7F09066
:08B67F0001F8F090023EF022F8
:10A3A700304E5275840190023FE0B40A005043904A
:10A3B700A3BDF828287302A3DB02A3DE02A3E102F0
:10A3C700A3E402A3E702A3EA02A3ED02A3F002A318
:10A3D700F302A3F602AFC702AEB002AF2102B61B6B
:10A3E70002B77602B42B02AA2802AF5902B5FB02C4
:06A3F700B75512B78622E3
:10AFC700E55B70317598989000A8E0B401131253AF
:10AFD7008CE49001F8F09001F7F090023F7403F0D1
:10AFE70022125389C252E49001F8F09001F7F090D1
:06AFF700023FE004F0221D
:10AEB0009000A8E01475F005A4B55B11E4B5F00DA1
:10AEC00075989812538C90023F7403F022E55B75DD
:10AED000F00584AFF0BF0110C253C2529001F87464
:09AEE00001F090023FE004F022B1
:10AF2100E55B75F00584AFF0BF042C20531EE55B93
:10AF310075F00584FF248DF582E43401F583E4F096
:10AF410074A22FF582E43401F583E4F0E49001F872
:08AF5100F090023FE014F02231
:10B61B009000A8E075F005A424FDB55B11758401BD
:0FB62B009000A9E0F599C25290023FE004F0228E
:10B776007584019000AAE0F59990023FE004F0225A
:10B42B009000A8E0FFB4140790023F7406F022EFDF
:10B43B0075F005A4B55B14E4B5F0101253899002B6
:0CB44B003FE004F0C252E49001F8F0224F
:10AA2800E55B75F00584AFF0BF0111C253C25290C7
:10AA380001F87401F090023FE004F022E55BB46491
:10AA48001F12538990022CE0700B9001F8F09002CD
:10AA58003F7408F022E49001F8F090023F7409F086
:01AA680022CB
:10AF5900E55B75F00584AFF0BF042C20531EE55B5B
:10AF690075F00584FF248DF582E43401F583E4F05E
:10AF790074A22FF582E43401F583E4F0E49001F83A
:08AF8900F090023FE014F022F9
:10B5FB00E55BB4651A756D01756E01756FFFE490AF
:10B60B00022AF090023F7409F09001F87402F022C4
:10B75500E55BB4690BC24EE49001F8F090023FF04E
:01B7650022C1
:10B78600C24EE49001F8F09001F7F090023FF022EB
:10745200789DE660011678A3E6600116900000E0D0
:10746200600214F0900002E0600214F0900001E06B
:10747200600214F0900003E0600214F0900004E057
:10748200600214F0900010E0600214F090000FE02F
:10749200600214F0900253E0600214F090025CE08B
:1074A200600214F0789F16E66003027591789F7669
:1074B2000A789EE6600116E54260021542900005D8
:1074C200E0600214F0900006E0600214F090000701
:1074D200E0600214F0900008E0600214F0900009ED
:1074E200E0600214F090000AE0600214F090000BD9
:1074F200E0600214F090000DE0600214F090000EC3
:10750200E0600214F0900256E0600214F078A4E603
:1075120060011690026CE0600214F090026FE0606D
:107522000214F0900270E0600214F078A016E67087
:107532005E78A0760A900012E0600214F078A6E667
:107542001846600708E6161870011690025DE060A2
:107552000214F090025EE0600214F090026AE060B1
:107562000214F0900272E0600214F078A116E67044
:107572001E78A1760A900013E0600214F078A21639
:10758200E6700C78A27606900011E0600214F022F8
:10809400535155452020434F53202053454E5345BB
:1080A400004F4E202020202020202020202020208F
:1080B40020004F4646202020202020202020202061
:1080C4002020002424242424242424242424242498
:1080D400242424242424242424242424242424245C
:1080E400242424242424242424242424242424244C
:1080F400242424231A1B1C1D1E1F20212224242473
:1081040024242424000102030405060708090A0B99
:108114000C0D0E0F10111213141516171819242410
:1081240024242424000102030405060708090A0B79
:108134000C0D0E0F101112131415161718192424F0
:1081440024242400000AAB0D55100012AB15551859
:10815400001AAB1D55200022AB255528002AAB2D53
:0D81640055300032AA355538003AAA3D5575
:10B56E00751F01E51FC394155018AF1F74B62FF544
:10B57E0082E43401F583E0FFEF60037F0122051FB3
:04B58E0080E17F00D9
:01B592002296
:10A2F800205455128668EF6401704D900119E0FFF3
:10A30800EF24FF92499001F6E0FF74E02FF582E414
:10A318003401F583E0FF9001F9EFF09001F6E0FFDA
:10A3280074CB2FF582E43401F583E0FF9001FAEF56
:10A33800F09001F6E0FF9001FBEFF01256FA900161
:09A34800FCEFF0128D50D22D2221
:10866800900171E4F0A3E4F0900174E4F0A3E4F065
:10867800900170E4F0900170E0FFEFC3941540039F
:1086880002870C9001F6E0FFEFD3941440069001A6
:10869800F67401F09001F6E0FF74B62FF582E43429
:1086A80001F583E0FF900173EFF0900173E0FFEFB5
:1086B800B401159001F6E0FF74B62FF582E4340199
:1086C800F5837402F07F0122900173E0FFEFB4029A
:1086D80024900171E0FEA3E0FFEF4E701890017145
:1086E800E4F0A37401F09001F6E0FF7E00900174BD
:1086F800EEF0A3EFF09001F6E004F0900170E004D2
:10870800F002867D900171E0FEA3E0FFEF4E700459
:108718007F002222900175E0FF9001F6EFF07F01C3
:01872800222E
:1084D000900171E4F0A3E4F0900174E4F0A3E4F0FF
:1084E000900170E4F0900170E0FFEFC39415400339
:1084F0000285819001F6E0FFEFD3941440069001CD
:10850000F67401F09001F6E0FF74B62FF582E434C2
:1085100001F583E0FF900173EFF0900173E0FFEF4E
:1085200060509000A8E0FF9001F6E0FEEE6F604220
:10853000900173E0FFEFB401159001F6E0FF74B60F
:108540002FF582E43401F5837402F07F012290015B
:1085500071E0FEA3E0FFEF4E70189001F6E0FF7EA1
:1085600000900174EEF0A3EFF0900171E4F0A374B9
:1085700001F09001F6E004F0900170E004F0028454
:10858000E5900171E0FEA3E0FFEF4E70047F002252
:0E85900022900175E0FF9001F6EFF07F0122CE
:1056FA009000A8E0FFEFD3941440037F2022900388
:10570A0073E4F0900372E4F09000A8E0FF90037055
:10571A00EFF0900114E0FFEFD3940650030257EE26
:10572A00900371E4F0900371E0FFEFC39415400316
:10573A000257E7900370E0FFEFB415069003707408
:10574A0001F0900370E0FF748C2FF582E43401F5C8
:10575A0083E0FFEF64FF7076900370E0FF74472FD9
:10576A00F582E43401F583E0FF9000A8E0FE744777
:10577A002EF582E43401F583E0FEEEC39F404F909C
:10578A0000A8E0FF900370E0FEEEB50706900370F4
:10579A00E0FF22900370E0FF74472FF582E43401A2
:1057AA00F583E0FF900372E0FEEFD39E4020900362
:1057BA0070E0FF900373EFF0900370E0FF74472FDF
:1057CA00F582E43401F583E0FF900372EFF0900371
:1057DA0071E004F0900370E004F002572F90037315
:1057EA00E0FF2222900371E4F0900371E0FFEFC31F
:1057FA00941540030258AA900370E0FFEF700690D8
:10580A0003707414F0900370E0FF748C2FF582E437
:10581A003401F583E0FFEF64FF7076900370E0FFD8
:10582A0074472FF582E43401F583E0FF9000A8E085
:10583A00FE74472EF582E43401F583E0FEEEC39F41
:10584A00404F9000A8E0FF900370E0FEEEB5070617
:10585A00900370E0FF22900370E0FF74472FF582F7
:10586A00E43401F583E0FF900372E0FEEFD39E403B
:10587A0020900370E0FF900373EFF0900370E0FF55
:10588A0074472FF582E43401F583E0FF900372EF49
:10589A00F0900371E004F0900370E014F00257F303
:0558AA00900373E0FF14
:0158AF0022D6
:1058B0009000A8E0FFEFD3941440037F20229003D0
:1058C00077E4F0900376E4F0900114E0FFEFD394D6
:1058D0000650030259959000A8E0FFEF04FF9003E3
:1058E00074EFF0900375E4F0900375E0FFEFC3945C
:1058F00015400302598E900374E0FFEFD3941440D7
:10590000069003747401F0900374E0FF748C2FF51B
:1059100082E43401F583E0FFEF64FF70629003746A
:10592000E0FF74472FF582E43401F583E0FF900037
:10593000A8E0FE74472EF582E43401F583E0FEEE24
:10594000C39F403B900374E0FF74472FF582E4341B
:1059500001F583E0FF900376E0FEEFD39E402090B8
:105960000374E0FF900377EFF0900374E0FF744757
:105970002FF582E43401F583E0FF900376EFF09099
:105980000375E004F0900374E004F00258E890031B
:1059900077E0FF22229000A8E0FFEF14FF9003744D
:1059A000EFF0900375E4F0900375E0FFEFC39415FA
:1059B0004003025A4A900374E0FFEF7006900374AC
:1059C0007414F0900374E0FF748C2FF582E43401BA
:1059D000F583E0FFEF64FF7062900374E0FF7447AB
:1059E0002FF582E43401F583E0FF9000A8E0FE7417
:1059F000472EF582E43401F583E0FEEEC39F403B81
:105A0000900374E0FF74472FF582E43401F583E0DE
:105A1000FF900376E0FEEFD39E4020900374E0FFFA
:105A2000900377EFF0900374E0FF74472FF582E462
:105A30003401F583E0FF900376EFF0900375E00406
:0F5A4000F0900374E014F00259A7900377E0FF91
:015A4F002234
:10B708009000A8E0FFEFD3941440037F202290001C
:04B71800A8E0FF2284
:1076CB009001F5E0FFEFD3941440069001F574019F
:1076DB00F0900170E4F09001F5E0FF74CB2FF58290
:1076EB00E43401F583E0FF9001F5E0FE74A12EF583
:1076FB0082E43401F583E0FEEEB507269001F5E058
:10770B00FF74E02FF582E43401F583E0FF9001F57F
:10771B00E0FE748C2EF582E43401F583E0FEEE6F0F
:10772B0060069001707401F09001F5E0FF748C2FEE
:10773B00F582E43401F583E0FF9000A8E0FEEF6EE4
:10774B00600E9000A8E0FF9001F5E0FEEE6F703A3E
:10775B00900170E0FFEF60439001F5E0FFEFD394F1
:10776B001550149001F5E0FF74B62FF582E4340147
:10777B00F5837401F080249001F5E0FF74B62FF5CA
:10778B0082E43401F583E4F080119001F5E0FF749D
:10779B00B62FF582E43401F583E4F0900170E0FF3D
:1077AB00EF60449001F5E0FF74A12FF582E4340102
:1077BB00F583E0FF9001F5E0FE74CB2EF582E43407
:1077CB0001F583EFF09001F5E0FF748C2FF582E467
:1077DB003401F583E0FF9001F5E0FE74E02EF582B5
:0E77EB00E43401F583EFF09001F5E004F022A4
:106C5000900239E0FFEF6003026D0B90000BE0FF44
:106C6000EF70037F012212A9E6EFB4010312009630
:106C700012A9E6EF70031200562046037F0022128D
:106C8000A9E6EF64016003026D0B30467BC246202B
:106C900036092037062038031270639000A4E0FF05
:106CA000900235EFF09000A5E0FF900236EFF090F3
:106CB00000A3E0FF900237EFF0900237E0FFEFB45F
:106CC0001F14900233E0FF900236E0FEEEB5070697
:106CD0001200567F0122900232E0FF900235E0FE62
:106CE000EEB5070E900233E0FF900236E0FEEE6F45
:106CF00060099002397401F07F002290010BE0FFDF
:106D000090000BEFF07F00227F0022900239E0FF1D
:106D1000EF64016003026DAD90000BE0FFEF7003C4
:106D20007F012212A9E6EFB4010312009612A9E630
:106D3000EF70031200562046037F0022C2461270F5
:106D4000639000A4E0FF900235EFF09000A5E0FF13
:106D5000900236EFF09000A3E0FF900237EFF09042
:106D60000237E0FFEFB41F14900233E0FF900236C9
:106D7000E0FEEEB507061200567F0122900232E0D7
:106D8000FF900235E0FEEEB50720900233E0FF9061
:106D90000236E0FEEEB5071290010BE0FF90000B0B
:106DA000EFF0900239E4F07F00227F00227F002282
:10A9E600900102E0FFEF600D12538F40047F01805B
:10A9F600027F002222900103E0FFEF601390010422
:10AA0600E0FFE532D39F40047F0122227F0022220D
:10AA1600900104E0FFE532C39F50047F0122227FAC
:02AA260000220C
:109DB700900170E4F0900170E0FFEFC3940A5058EF
:109DC700900170E0FF74262FF582E43401F583E0FB
:109DD700FFEFB42013900170E0FF743E2FF582E48B
:109DE7003401F5837426F022900170E0FF74262F6A
:109DF700F582E43401F583E0FFEF9080C793FF908D
:109E07000170E0FE743E2EF582E43401F583EFF035
:099E1700900170E004F0809D222E
:1068260090023BE0FFEF60030268DC90000DE0FFA2
:10683600EF70037F012212A9E6EFB401031200965E
:1068460012A9E6EF700312005690023AE0FFEFB489
:1068560001062022037F002290023AE0FFEFB402F5
:1068660006202F037F002212A9E6EF6401706490D0
:10687600023AE0FFEF6401702130221EC222E54F8A
:10688600654E600990023B7401F07F002290011072
:10689600E0FF90000DEFF07F002290023AE0FFEF5C
:1068A6006402702F302F2CC22F90023DE544F090E9
:1068B600023DE0FF90023CE0FEEE6F600990023B75
:1068C6007401F07F0022900110E0FF90000DEFF0C0
:1068D6007F00227F002290023BE0FFEF640160030D
:1068E60002698990000DE0FFEF70037F012212A973
:1068F600E6EFB4010312009612A9E6EF7003120048
:106906005690023AE0FFEFB401062022037F0022F0
:1069160090023AE0FFEFB40206202F037F00221216
:10692600A9E6EF6401705A90023AE0FFEFB4011C49
:10693600302219C222E54FB54E1290023BE4F09088
:106946000110E0FF90000DEFF07F002290023AE088
:10695600FFEF6402702B302F28C22F90023DE544D2
:10696600F090023DE0FF90023CE0FEEEB50712908B
:10697600023BE4F0900110E0FF90000DEFF07F0085
:04698600227F00224A
:10B28F008F7A9000F5E0FF8F36AF7AEF3395E0FEBF
:10B29F00EF25E0FFEE33FE74472FF58274813EF504
:0FB2AF0083E493F508740193F509D229D20C2298
:109EEF007BFF7A80799412ABEC12538F400B7BFF80
:109EFF007A8079A512A61280097BFF7A8079B61233
:109F0F00A6127F17127D63AF321254289000CBE058
:109F1F00FF127D319000CCE0FF127D319000CDE03B
:109F2F00FF127D317F1C127D63AF311254289000D8
:109F3F00CBE0FF127D319000CCE0FF127D3190001D
:079F4F00CDE0FF127D31227D
:0BB80B007508027509ABD229D20C228F
:0BB8160075081A7509ABD229D20C226C
:10B3D200900107E0FFEF6013900108E0FFE531D331
:10B3E2009F40047F0122227F002222900108E0FF79
:0DB3F200E531C39F50047F0122227F00221D
:10B2BE008F7B9000F7E0FF8F36AF7BEF3395E0FE8C
:10B2CE00EF25E0FFEE33FE74472FF58274813EF5D5
:0FB2DE0083E493F508740193F509D229D20C2269
:05001600C229C20C220A
:0C0096009000FEE0FF8F34D208C2092267
:05005600D208D20922CE
:10B79600900102E0FFEF600412952E2212698A22C0
:10952E00900245E0FFEF701612538F4072900105C6
:10953E00E0FF90000FEFF0900245E004F022900261
:10954E0045E0FFEF6401702812538F401C90000F0E
:10955E00E0FFEF704AD25C90010FE0FF90000CEF3D
:10956E00F0900245E004F02222900245E4F022221F
:10957E00900245E0FFEFB4022112538F400B900191
:10958E000FE0FF90000CEFF02290000CE0FFEF7068
:10959E000EC25C900245E4F02222900245E4F022D5
:10698A00900245E0FFEF704C900103E0FFEF6023B7
:10699A00900104E0FFE532D39F4013900105E0FF28
:1069AA0090000FEFF0900245E004F0228026C25CCE
:1069BA00228021900104E0FFE532C39F5013900129
:1069CA0005E0FF90000FEFF09002457403F022807B
:1069DA0003C25C22900245E0FFEF6401703590012A
:1069EA0004E0FFEF24FBFFE532D39F401F90000F26
:1069FA00E0FFEF6003026AEDD25C900106E0FF90CF
:106A0A000010EFF0900245E004F02222900245E4E3
:106A1A00F02222900245E0FFEF6402702E900104FA
:106A2A00E0FFEF24FBFFE532D39F400B900106E025
:106A3A00FF900010EFF022900010E0FFEF600302D9
:106A4A006AEDC25C900245E4F02222900245E0FF22
:106A5A00EF64037043900104E0FF7E00EF2405FF1A
:106A6A00EE3400FEAD327C00C3ED9FEE6480F8EC9C
:106A7A00648098501C90000FE0FFEF7066D25C9023
:106A8A000106E0FF900010EFF0900245E004F022CA
:106A9A0022900245E4F02222900245E0FFEF6404CE
:106AAA00703C900104E0FF7E00EF2405FFEE340005
:106ABA00FEAD327C00C3ED9FEE6480F8EC648098F2
:106ACA00500B900106E0FF900010EFF022900010AA
:106ADA00E0FFEF700EC25C900245E4F022229002C1
:046AEA0045E4F0226D
:101F0400202020464C4558204949492020202020A3
:101F14000020202020202020202020202049444C64
:101F240045004E4F204C54522042555320204944E2
:101F34004C45002054657374696E67204D6F646569
:101F44002020200043726F73732042757379204DF3
:101F54006F6465310043726F737320427573792027
:101F64004D6F6465320043726F73732042757379E9
:101F7400204D6F6465330043726F73732042757331
:101F840079204D6F6465340050726F6772616D6DB6
:101F9400696E6757726F6E6700435443535320361C
:101FA400332E302020202020204354435353203606
:101FB400372E3020202020202043544353532036F2
:101FC400392E3420202020202043544353532037DB
:101FD400312E3920202020202043544353532037CE
:101FE400342E3420202020202043544353532037C0
:101FF400372E3020202020202043544353532037B1
:10200400392E372020202020204354435353203896
:10201400322E35202020202020435443535320388F
:10202400352E34202020202020435443535320387D
:10203400382E352020202020204354435353203968
:10204400312E35202020202020435443535320395F
:10205400342E382020202020204354435353203949
:10206400372E342020202020204354435353203142
:1020740030302E302020202020435443535320312D
:1020840030332E3520202020204354435353203115
:1020940030372E3220202020204354435353203104
:1020A40031302E39202020202043544353532031F3
:1020B40031342E38202020202043544353532031E0
:1020C40031382E38202020202043544353532031CC
:1020D40032332E30202020202043544353532031C8
:1020E40032372E33202020202043544353532031B1
:1020F40033312E38202020202043544353532031A1
:1021040033362E352020202020435443535320318E
:1021140034312E3320202020204354435353203184
:1021240034362E3220202020204354435353203170
:1021340035312E3420202020204354435353203162
:1021440035362E372020202020435443535320314A
:1021540035392E3820202020204354435353203136
:1021640036322E3220202020204354435353203132
:1021740036352E352020202020435443535320311C
:1021840036372E3920202020204354435353203106
:1021940037312E3320202020204354435353203101
:1021A40037332E38202020202043544353532031EA
:1021B40037372E33202020202043544353532031DB
:1021C40037392E39202020202043544353532031C3
:1021D40038332E35202020202043544353532031BC
:1021E40038362E32202020202043544353532031AC
:1021F40038392E3920202020204354435353203192
:1022040039322E3820202020204354435353203188
:1022140039362E3620202020204354435353203176
:1022240039392E3520202020204354435353203263
:1022340030332E3520202020204354435353203262
:1022440030362E352020202020435443535320324F
:1022540031302E3720202020204354435353203242
:1022640031382E3120202020204354435353203230
:1022740032352E372020202020435443535320321C
:1022840032392E312020202020435443535320320E
:1022940033332E36202020202043544353532032FE
:1022A40034312E38202020202043544353532032ED
:1022B40035302E33202020202043544353532032E2
:1022C40035342E31202020202020202020202020C2
:1022D400202020202020202020444353203030364A
:1022E40020494E5620303231204443532030303779
:1022F40020494E5620323134204443532030313566
:1023040020494E5620313431204443532030313754
:1023140020494E562030353020444353203032314A
:1023240020494E5620303036204443532030323337
:1023340020494E5620303437204443532030323520
:1023440020494E5620323434204443532030323610
:1023540020494E5620343634204443532030333100
:1023640020494E56203632372044435320303332EE
:1023740020494E56203035312044435320303336E3
:1023840020494E56203137322044435320303433D1
:1023940020494E56203434352044435320303437BA
:1023A40020494E56203032332044435320303530B8
:1023B40020494E56203031372044435320303531A4
:1023C40020494E5620303332204443532030353395
:1023D40020494E562034353220444353203035347E
:1023E40020494E562034313320444353203036356F
:1023F40020494E5620323731204443532030373160
:1024040020494E562033303620444353203037324F
:1024140020494E562032343520444353203037333C
:1024240020494E562035303620444353203037342B
:1024340020494E562031373420444353203131341F
:1024440020494E5620373132204443532031313510
:1024540020494E5620313532204443532031313601
:1024640020494E56203735342044435320313232EC
:1024740020494E56203232352044435320313235E0
:1024840020494E56203336352044435320313331CE
:1024940020494E56203336342044435320313332BE
:1024A40020494E56203534362044435320313334AA
:1024B40020494E56203232332044435320313431A4
:1024C40020494E5620303135204443532031343393
:1024D40020494E5620343132204443532031343580
:1024E40020494E562032373420444353203135326C
:1024F40020494E562031313520444353203135355F
:1025040020494E5620373331204443532031353649
:1025140020494E562032363520444353203136323A
:1025240020494E562035303320444353203136352C
:1025340020494E562032353120444353203137321E
:1025440020494E562030333620444353203137340B
:1025540020494E56203037342044435320323035FE
:1025640020494E56203236332044435320323132F0
:1025740020494E56203335362044435320323134DB
:1025840020494E56203030372044435320323233D2
:1025940020494E56203133342044435320323235BF
:1025A40020494E56203132322044435320323236B1
:1025B40020494E56203431312044435320323433A1
:1025C40020494E562033353120444353203234348D
:1025D40020494E562030323520444353203234357E
:1025E40020494E562030373220444353203234366B
:1025F40020494E562035323320444353203235315E
:1026040020494E562031363520444353203235324A
:1026140020494E5620343632204443532032353537
:1026240020494E5620343436204443532032363128
:1026340020494E5620373332204443532032363318
:1026440020494E562032303520444353203236350B
:1026540020494E56203135362044435320323636F5
:1026640020494E56203435342044435320323731E8
:1026740020494E56203036352044435320323734D7
:1026840020494E56203134352044435320333036CC
:1026940020494E56203037312044435320333131C2
:1026A40020494E56203636342044435320333135A6
:1026B40020494E562034323320444353203332359C
:1026C40020494E562035323620444353203333318B
:1026D40020494E5620343635204443532033333278
:1026E40020494E5620343535204443532033343367
:1026F40020494E5620353332204443532033343658
:1027040020494E562036313220444353203335314C
:1027140020494E5620323433204443532033353637
:1027240020494E562032313220444353203336342C
:1027340020494E562031333120444353203336351B
:1027440020494E562031323520444353203337310B
:1027540020494E56203733342044435320343131FA
:1027640020494E56203232362044435320343132ED
:1027740020494E56203134332044435320343133DE
:1027840020494E56203035342044435320343233CC
:1027940020494E56203331352044435320343331BD
:1027A40020494E56203732332044435320343332A9
:1027B40020494E5620353136204443532034343595
:1027C40020494E5620303433204443532034343689
:1027D40020494E5620323535204443532034353277
:1027E40020494E5620303533204443532034353469
:1027F40020494E5620323636204443532034353552
:1028040020494E5620333332204443532034363249
:1028140020494E5620323532204443532034363436
:1028240020494E5620303236204443532034363526
:1028340020494E5620333331204443532034363616
:1028440020494E5620363632204443532035303307
:1028540020494E56203136322044435320353036F9
:1028640020494E56203037332044435320353136E7
:1028740020494E56203433322044435320353233DA
:1028840020494E56203234362044435320353236C4
:1028940020494E56203332352044435320353332B9
:1028A40020494E56203334332044435320353436A4
:1028B40020494E5620313332204443532035363597
:1028C40020494E5620373033204443532036303687
:1028D40020494E562036333120444353203631327A
:1028E40020494E5620333436204443532036323464
:1028F40020494E5620363332204443532036323753
:1029040020494E562030333120444353203633314E
:1029140020494E5620363036204443532036333235
:1029240020494E5620363234204443532036353421
:1029340020494E5620373433204443532036363210
:1029440020494E56203436362044435320363634FC
:1029540020494E56203331312044435320373033FD
:1029640020494E56203536352044435320373132E2
:1029740020494E56203131342044435320373233DA
:1029840020494E56203433312044435320373331C9
:1029940020494E56203135352044435320373332B5
:1029A40020494E56203236312044435320373334A5
:1029B40020494E5620333731204443532037343393
:1029C40020494E562036353420444353203735347D
:1029D40020494E5620313136204284A4830124C339
:1029E400040274A344C282E364D4430381231463C2
:0F29F40094B4C47D3D1D0D0585C5E5F5FD009529
:10792000900132E0FFB4010A9000A974FFF0E40274
:1079300079EDEF640260030279F21253617880E618
:1079400060030279E13054030279E1900238E0707B
:1079500032D22D900119E024FF92499000A8E0FF57
:107960009001F9F0900117E09001FAF09001FBEF1F
:10797000F01258B09001FCEFF0128D509002387464
:1079800002F0221284D0EF64017050D22D9001F6E3
:10799000E0FF24E0F582E43401F583E09001F9F0A2
:1079A00074CB2FF582E43401F583E09001FAF09076
:1079B00001F6E09001FBF01256FA9001FCEFF09016
:1079C00001F9E0245BF582E43401F583E024FF92C1
:1079D00049128D50900238E014F022900238E014E1
:1079E000F09000A8E09000A9F0900117E09000AAA4
:1079F000F02290022DE0B40B005046907A02F82855
:107A00002873027A23027A26027A29027A2C027AD1
:107A10002F027A32027A41027A35027A38027A3BB0
:107A2000027A3E022A030271BA02730D0241B102C8
:107A3000997102321C02B7B502B7C402B7D302B7BC
:077A4000E2E490022DF022A8
:102A03009000A8E0D39414400302321B90022EE0FE
:102A1300B40C004003023216902A22F828287302CD
:102A23002A46022A5E022C9B022CE2022CFF022D74
:102A330030022E06022E8E022F21022F6002302A30
:102A43000231177BFF7A1F790412ABEC7BFF7A1FED
:102A5300791512A61290022E022C9720552390026C
:102A63006AE0701D204F127BFF7A1F790412ABECD2
:102A73007BFF7A1F792612A61290026A7402F0C2B3
:102A83004F20A55C125361900133E0600312536D34
:102A9300900130E0900000F09000A8E0FF9000A9C2
:102AA300F0900117E0FE9000AAF090022E7405F05A
:102AB3009001F9EFF09001FAEEF09000A8E0900198
:102AC300FBF01256FA9001FCEFF0900119E024FF9D
:102AD3009249128D50D22D7BFF7A1F793702ABECCE
:102AE30012A9E6EF6401705C304659C2469000A417
:102AF300E0FFC39415504D745B2FF582E43401F568
:102B030083E0FFA244E4336F703A127063A24492ED
:102B1300459000A4E0900232F09000A5E0900233CB
:102B2300F09000A3E0900234F0641F60179002322B
:102B3300E0FF900233E0FD7C00128C0D90022D74B7
:102B430002023143C24612B56EBF011712536190A0
:102B53000133E0600312536D900130E0900000F008
:102B6300022F0B900134E0601C12A9E6EF640160B0
:102B73000612B3D2BF010E900111E078A4F69002C1
:102B83002E7409F02212A9E6EF640170683022283E
:102B9300C22290023A04F0D220854E4FE54F75F0E1
:102BA30010A4249DF9741F35F0FA7BFF12ABECAF30
:102BB3004F1291F6C220802A302F3AC22F90023C46
:102BC300E544F075F010A424DDF9742235F0FA7BA6
:102BD300FF12ABEC90023CE0FF12904390023A7478
:102BE30002F090022D7405F0E490022EF090011192
:102BF300E078A4F622C222C22F78A6E618467030E7
:102C0300900118E0FF6029760008A6079000A974D8
:102C1300FFF09000AAF0125361900133E0600312B9
:102C2300536D900130E0900000F090022E0231A528
:102C3300900123E0FF700302321B900011E0600358
:102C430002321B900121E0FE6010700302321B90E0
:102C53000240E06401600302321B900011EFF0E4D4
:102C6300900240F0125361900133E0600312536D00
:102C7300900130E0900000F09000A8E09000A9F0EF
:102C83009000AA74FDF0E490022EF0900122E090EF
:102C9300022D60647401F022900000E060030232B0
:102CA3001B30540302321B9000A8E0FF9001F9F09F
:102CB3009001FA74FFF09001FBEFF09001FCF090AB
:102CC3000119E024FF9249128D50D22D203609209C
:102CD300370620380312710590022E7403F0227810
:102CE30080E6600302321B30540302321B90010C56
:102CF300E0900001F090022E7404F022900001E0B5
:102D0300600302321B125367900133E060031253D6
:102D130073E490022EF090024004F020360C20372A
:102D230009203806127D80127D92022DFB30A50307
:102D3300022DF69000A8E09000A9F0900117E09012
:102D430000AAF012A9E6BF01051200968003120043
:102D5300567880E6600302321B30540302321B9024
:102D63000238E07034D22D900119E024FF9249908B
:102D730000A8E0FF9001F9F0900117E09001FAF04C
:102D83009001FBEFF01258B09001FCEFF0128D5060
:102D93009002387402F00271051284D0EF6401705E
:102DA3004FD22D9001F6E0FF24E0F582E43401F5E3
:102DB30083E09001F9F074CB2FF582E43401F583BD
:102DC300E09001FAF09001F6E09001FBF01256FA60
:102DD3009001FCEFF09001F9E0245BF582E434010B
:102DE300F583E024FF9249128D501271050231FAE6
:102DF3000231FAE490022EF09000A974FFF09000E3
:102E0300AAF022900000E0600302321B3054030258
:102E1300321B7880E6600302321B9000A974FFF036
:102E23009000AAF0128668EF64016003022F1290EB
:102E330001F6E0FF24E0F582E43401F583E090013C
:102E4300F9F074CB2FF582E43401F583E09001FAB5
:102E5300F09001F6E09001FBF012B7089001FCEF4F
:102E6300F09001F9E0245BF582E43401F583E0247A
:102E7300FF9249128D50D22D203609203706203873
:102E83000312710590022E7407F02212A9E6EF6473
:102E930001705F30465EC2469000A4E0FFC3941504
:102EA3005052745B2FF582E43401F583E0FFA244B2
:102EB300E4336F703F127063A24492459000A4E024
:102EC300900232F09000A5E0900233F09000A3E06E
:102ED300900234F0641F601C900232E0FF900233D2
:102EE300E0FD7C00128C0DE490022EF090022D0286
:102EF30031A5C2467880E6600302321B30540302D8
:102F0300321B12B56EEF600790022E7406F022900A
:102F1300010CE0900001F090022E7408F022900062
:102F230001E0600302321B125367900133E0600338
:102F33001253739002407401F0E490022EF090005B
:102F4300A974FFF09000AAF030360302321B303729
:102F53000302321B30380302321B027D9212A9E6B0
:102F6300EF64017063304660C2469000A4E0FFC383
:102F730094155054745B2FF582E43401F583E0FF1C
:102F8300A244E4336F7041A24492459000A4E090C0
:102F93000232F09000A5E0900233F09000A3E0909D
:102FA3000234F0127063900234E0641F601A9002DE
:102FB30032E0FF900233E0FD7C00128C0DE49002BE
:102FC3002EF090022D0231A5C24678A4E6600302DA
:102FD300321B9000A8E09000A9F09000AA74FDF0C5
:102FE300900134E0FF64016004EFB4021512A9E616
:102FF300BF010F900112E090000AF090022E740AB4
:10300300F022900134E0FF64036004EFB40415126E
:10301300B3D2BF010F900112E090000AF090022E8C
:10302300740BF02202321612A9E6BF0108900112B6
:10303300E090000AF090000AE0701B1253679001C1
:1030430018E0FF78A5760008A6079000A974FFF0A2
:103053009000AA023143900134E0B401097BFF7A66
:103063001F79480231541253617BFF7A1F79591239
:10307300A6127880E6600302320730540302320757
:10308300900238E07031D22D900119E024FF92496B
:103093009000A8E0FF9001F9F0900117E09001FA89
:1030A300F09001FBEFF01258B09001FCEFF0128D9D
:1030B300509002380231A51284D0EF6401704CD2D3
:1030C3002D9001F6E0FF24E0F582E43401F583E07E
:1030D3009001F9F074CB2FF582E43401F583E0908D
:1030E30001FAF09001F6E09001FBF01256FA90011C
:1030F300FCEFF09001F9E0245BF582E43401F58301
:10310300E024FF9249128D500231FA900238E01404
:10311300F002320712B3D2BF0108900112E090000F
:103123000AF090000AE0701C125367900118E0FF48
:1031330078A5760008A6079000A974FFF09000AA6E
:10314300F0023216900134E0B403097BFF7A1F7951
:103153006A02A6127BFF7A1F797B12A612125361B1
:103163007880E6600302320730540302320790028C
:1031730038E07032D22D900119E024FF924990007B
:10318300A8E0FF9001F9F0900117E09001FAF090A8
:1031930001FBEFF01258B09001FCEFF0128D50904C
:1031A30002387402F0221284D0EF64017050D22DE1
:1031B3009001F6E0FF24E0F582E43401F583E0902A
:1031C30001F9F074CB2FF582E43401F583E090012B
:1031D300FAF09001F6E09001FBF01256FA9001FC30
:1031E300EFF09001F9E0245BF582E43401F583E02C
:1031F30024FF9249128D50900238E014F02290027D
:1032030038E014F09000A8E09000A9F09000AA74B0
:09321300FDF022E490022EF022ED
:1071BA0090022EE0FF700F900000E0600302730C53
:1071CA0090022F027306EF6401705F12A2F8900218
:1071DA002FE0D39409400990010CE090000180202F
:1071EA0090022FE0FF04F0743E2FF582E43401F59B
:1071FA0083E0900231F0E0FFB4260D900001743272
:10720A00F090022E7406F022EFB4240A900124E0D2
:10721A0075F0060272BF900231E09029DD93900268
:10722A0031F05407900230F0807D90022EE0640223
:10723A00703912A2F8900124E0FF900002F0900247
:10724A0031E0FE30E709EF75F003A4900002F0EE9A
:10725A0025E0900231F0900230E014F0900125E030
:10726A00FF12B2BE90022E7403F02290022EE0B4F6
:10727A00031E12A2F8900002E0600302730C900150
:10728A0024E0900002F012001690022E7404F022FC
:10729A0090022EE06404702912A2F8900002E070B5
:1072AA0061900230E0600790022E7402F022900191
:1072BA0024E075F003A4900002F090022E7405F009
:1072CA002290022EE0B4050B12A2F8900002E070A0
:1072DA0031802A90022EE0B40628900001E0702244
:1072EA00125367900133E06003125373900118E060
:1072FA00FF78A5760008A607E490022DF090022EEA
:03730A0004F0226A
:10730D0090022EE0704F9000E5E0604212536190C4
:10731D000133E0600312536D900130E0900000F0F6
:10732D009000E6E060229000E9E0B4300F9000E8B4
:10733D00E0B430089000E7E064306012206A0FD2AC
:10734D006A90022D7407F02290022D0273DF9002D5
:10735D002E7404F02290022EE0640170487880E6CD
:10736D006003027451305403027451900232E09064
:10737D0001F9F0900233E09001FAF09001FB741FD7
:10738D00F01256FA9001FCEFF0A2459249128D5081
:10739D00D22D2036092037062038031271059002B0
:1073AD002E7402F02290022EE0640270297880E69D
:1073BD00600302745130540302745190010CE0903B
:1073CD000001F0203609203706203803127D9290F7
:1073DD00022E7403F02290022EE0640370359000AB
:1073ED0001E07060125367900133E0600312537334
:1073FD00900118E0FF78A5760008A607E490022D0D
:10740D00F07BFF7A1F790412ABEC7BFF7A1F7915A5
:10741D0002A61290022EE0D394034028E490022D90
:10742D00F090022E04F07BFF7A1F790412ABEC7BF7
:10743D00FF7A1F791512A612125367900133E0607F
:05744D0003125373223D
:1041B10090022EE0FF7017900232E09000A9F0907B
:1041C1000233E09000AAF090022E7401F022EF6415
:1041D10001705A900000E06003024586A2459249B1
:1041E100900232E09001F9F0900233E09001FAF090
:1041F1009000A8E09001FBF01258B09001FCEFF0A4
:10420100128D50D22D203609203706203803127125
:104211000590010BE090000BF090010DE090001271
:10422100F09002387408F090022E0242D790022ECC
:10423100E06402702F126C50EF600280467880E6D5
:1042410060030245863054030245867628D2549095
:104251000238E014F0E060030245867402F0900237
:104261002E04F02290022EE0640360030243411207
:104271006C50EF6002800C90010DE0600D90001217
:10428100E0700790022E7404F0227880E660030249
:104291004586305403024586900238E0703CA245C1
:1042A1009249900232E09001F9F0900233E09001DE
:1042B100FAF09000A8E09001FBF01258B09001FCD8
:1042C100EFF0128D50D22D20360920370620380309
:1042D1001271059002387402F0221284D0EF640149
:1042E10070579001F6E0FF24E0F582E43401F58394
:1042F100E09001F9F074CB2FF582E43401F583E00D
:104301009001FAF09001F6E09001FBF01256FA905C
:1043110001FCEFF09001F9E0245BF582E43401F552
:1043210083E024FF9249128D50D22D20360B203785
:10433100082038051271058000900238E014F0223F
:1043410090022EE0640470342036092037062038AC
:1043510003127D80120056E4900239F09000E4E0EF
:104361006014900131E0FF12B28F78A3761478A324
:10437100E670FB12B84B90022E7405F090022EE00D
:10438100640570457880E6704020543DA24592490D
:10439100900232E09001F9F0900233E09001FAF0DE
:1043A1009001FB741FF012B7089001FCEFF0128D21
:1043B100509002387403F020360920370620380364
:1043C10012710590022E7406F090022EE0FF640631
:1043D10070297880E67024205421900238E0700F13
:1043E10090010CE0900001F090022E7407F0227809
:1043F100807628D254900238E014F0EF640760030D
:10440100024586900134E0601F302209302F0612E8
:10441100B3D2EF7013E490022DF090022EF09001D0
:1044210011E078A4F602457A12A9E6EF640160036F
:104431000244B92046030244B9C24612A9E6EF6418
:104441000170759000A4E0FFC39415506B745B2F4D
:10445100F582E43401F583E0FFA244E4336F705840
:10446100A24492459000A4E0900232F09000A5E0B1
:10447100900233F09000A3E0900234F0641F6038A2
:10448100900232E0FFC39415502E745B2FF582E445
:104491003401F583E0FFA245E433B5071B900232F6
:1044A100E0FF900233E0FD7C00128C0D90022D7430
:1044B10002F0E490022EF0227880E67069205466C2
:1044C100128668EF6401705E9001F6E0FF24E0F56A
:1044D10082E43401F583E09001F9F074CB2FF58289
:1044E100E43401F583E09001FAF09001F6E09001E7
:1044F100FBF01256FA9001FCEFF09001F9E0245B19
:10450100F582E43401F583E024FF9249128D509045
:10451100022E7406F0E490022DF0203609203706B1
:10452100203803127105900001E070591253679011
:104531000133E06003125373203609203706203817
:1045410003127D929000A974FFF09000AAF09002EE
:10455100407401F0E490022DF090022E04F0203618
:10456100182037152038127BFF7A1F790412ABEC23
:104571007BFF7A1F791512A612900118E0FF78A52A
:06458100760008A60722E7
:1099710090022EE0FF7017900000E07065F559F538
:109981005A9000F8E0F53490022E7401F022EFB401
:10999100011D12A2F8D20B125DA55013E4F559C2B4
:1099A1000B90010CE0900001F090022E7402F090F7
:1099B100022EE06402702B12A2F8900001E07022E6
:1099C100125367900133E06003125373900118E062
:1099D100FF78A5760008A607E490022DF090022EEC
:0399E10004F0226D
:10321C0090022EE0600302333212A9E6EF640170D3
:10322C0057304654C2469000A4E0FFC39415504852
:10323C00745B2FF582E43401F583E0FFA244E433A0
:10324C006F7035127063A24492459000A4E0900216
:10325C0032F09000A5E0900233F09000A3E09002D1
:10326C0034F0641F6012900232E0FF900233E0FDF4
:10327C007C00128C0D02353BC24678A4E66003023A
:10328C00387412A9E6EF6401600302331E9000D972
:10329C00E07025125367900133E060031253739072
:1032AC000134E0B401109000A8E09000A9F0900067
:1032BC00AA74FEF080708066125361900133E06056
:1032CC000312536D900130E0900000F09000A8E0E4
:1032DC009000A9F09000AA74FEF09000DBE0601A58
:1032EC00206A09D26A90022D7409F0221253679059
:1032FC000133E06003125373802490010DE09000C1
:10330C0012F0900110E090000DF090022E7401F07C
:10331C008014125367900133E06003125373C22080
:10332C00E490022DF02290022EE06401600302333F
:10333C00CD900000E060030233CD90023AE06401CE
:10334C007036AF4F12962920367120376E20386BAD
:10335C00E54F75F010A4249DF9741F35F0FA7BFF2E
:10336C0012ABECE54F75F010A4249DF9741F35F0E9
:10337C00FA7BFF12A612804390023AE0640270417D
:10338C0090023CE0FF12188720363020372D203871
:10339C002A90023CE075F010A424DDF9742235F07B
:1033AC00FA7BFF12ABEC90023CE075F010A424DD2C
:1033BC00F9742235F0FA7BFF12A61290022E023815
:1033CC006E90022EE064027041126826EF601412B7
:1033DC007D8090022E7403F09000D7E070030238C9
:1033EC0074801E90010DE06021900012E0701B12A1
:1033FC007D8090022E7403F09000D7E070030238A9
:10340C007490011DE0900004F02290022EE0640301
:10341C006003023543900004E07048127D92120064
:10342C0056E490023BF09000D7E06014900131E03C
:10343C00FF12B28F78A3761978A3E670FB12B84B03
:10344C009000D8E0600F90011EE090000EF090020A
:10345C002E7404F02290011FE0900003F012B7F1DB
:10346C0002355F12A9E6EF6401705A12B7F13022EF
:10347C002CC22290023A7401F0C220854E4F2036A5
:10348C0019203716203813E54F75F010A4249DF938
:10349C00741F35F0FA7BFF12ABEC023593302F25FD
:1034AC00C22F90023CE544F0203617203714203808
:1034BC001175F010A424DDF9742235F0FA7BFF129B
:1034CC00ABEC0235BFC222C22F12A9E6EF64017029
:1034DC006430466112B7F1C220C2469000A4E0FFEE
:1034EC00C394155050745B2FF582E43401F583E0DE
:1034FC00FFA244E4336F703D127063A24492459076
:10350C0000A4E0900232F09000A5E0900233F0901D
:10351C0000A3E0900234F0641F601A900232E0FFC6
:10352C00900233E0FD7C00128C0DE490022EF090A2
:10353C00022D02386EC24690022EE0640460030233
:10354C00364790000EE0701112B7F190011FE09019
:10355C000003F090022E0237F412A9E6EF6401701A
:10356C006B12B7F1302230C22290023A7401F0850E
:10357C004E4FC220E54F75F010A4249DF9741F35F1
:10358C00F0FA7BFF12ABECAF4F1291F6E490022EE7
:10359C00F090022D0237F4302F32C22F90023CE50E
:1035AC0044F075F010A424DDF9742235F0FA7BFF99
:1035BC0012ABEC90023CE0FF12904390023A740282
:1035CC00F0E490022EF090022D0237F4C222C22FAA
:1035DC0012A9E6EF6401706130465E12B7F1C220A9
:1035EC00C2469000A4E0FFC39415504D745B2FF5B8
:1035FC0082E43401F583E0FFA244E4336F703A12A5
:10360C007063A24492459000A4E0900232F09000C6
:10361C00A5E0900233F09000A3E0900234F0641F18
:10362C006017900232E0FF900233E0FD7C00128CB8
:10363C000D90022D74020236C4C24690022EE06434
:10364C0005600302373D900003E0700790022E7472
:10365C0006F02212A9E6EF6401706430222BC2221C
:10366C0090023A04F0854E4FC220E54F75F010A43D
:10367C00249DF9741F35F0FA7BFF12ABECAF4F129F
:10368C0091F690022D7405802F302F33C22F9002AB
:10369C003CE544F075F010A424DDF9742235F0FA01
:1036AC007BFF12ABEC90023CE0FF12904390023A8D
:1036BC007402F090022D7405F0E490022EF022C2F8
:1036CC0022C22F12A9E6EF6401706430466112B772
:1036DC00F1C220C2469000A4E0FFC3941550507470
:1036EC005B2FF582E43401F583E0FFA244E4336FF1
:1036FC00703D127063A24492459000A4E090023297
:10370C00F09000A5E0900233F09000A3E09002341A
:10371C00F0641F601A900232E0FF900233E0FD7CEF
:10372C0000128C0DE490022EF090022D02386EC225
:10373C004690022EE064066003023874900001E0AB
:10374C00703D125367900133E060031253737BFF9B
:10375C007A1F790412ABEC7BFF7A1F791512A61233
:10376C00900118E0FF78A5760008A6079002407437
:10377C0001F0C220E490022DF090022E04F02212EF
:10378C00A9E6EF6401706530222CC22290023A0443
:10379C00F0854E4FE54F75F010A4249DF9741F353C
:1037AC00F0FA7BFF12ABECAF4F1291F6E490022EC5
:1037BC00F090022D8032302F33C22F90023CE54422
:1037CC00F075F010A424DDF9742235F0FA7BFF12A9
:1037DC00ABEC90023CE0FF12904390023A7402F082
:1037EC00E490022EF090022D7405F022C222C22F1A
:1037FC0012A9E6EF6401706E30466B12B7F1C2206D
:10380C00C2469000A4E0FFC39415505A745B2FF588
:10381C0082E43401F583E0FFA244E4336F70472067
:10382C003609203706203803127063A24492459063
:10383C0000A4E0900232F09000A5E0900233F090EA
:10384C0000A3E0900234F0641F601B900232E0FF92
:10385C00900233E0FD7C00128C0DE490022EF0906F
:09386C00022D7402F022C2462272
:0FB7B5007BFF7A1F798C12ABECE490022DF0220F
:0FB7C4007BFF7A1F798C12ABECE490022DF02200
:0FB7D3007BFF7A1F798C12ABECE490022DF022F1
:0FB7E2007BFF7A1F798C12ABECE490022DF022E2
:1045870043544353532036332E30202020202020FD
:1045970043544353532036372E30202020202020E9
:1045A70043544353532036392E34202020202020D3
:1045B70043544353532037312E39202020202020C5
:1045C70043544353532037342E34202020202020B7
:1045D70043544353532037372E30202020202020A8
:1045E70043544353532037392E372020202020208F
:1045F70043544353532038322E3520202020202087
:1046070043544353532038352E3420202020202074
:1046170043544353532038382E3520202020202060
:1046270043544353532039312E3520202020202056
:1046370043544353532039342E3820202020202040
:1046470043544353532039372E3420202020202031
:104657004354435353203130302E30202020202024
:104667004354435353203130332E3520202020200C
:104677004354435353203130372E322020202020FB
:104687004354435353203131302E392020202020EA
:104697004354435353203131342E382020202020D7
:1046A7004354435353203131382E382020202020C3
:1046B7004354435353203132332E302020202020BF
:1046C7004354435353203132372E332020202020A8
:1046D7004354435353203133312E38202020202098
:1046E7004354435353203133362E35202020202086
:1046F7004354435353203134312E3320202020207C
:104707004354435353203134362E32202020202067
:104717004354435353203135312E34202020202059
:104727004354435353203135362E37202020202041
:104737004354435353203135392E3820202020202D
:104747004354435353203136322E32202020202029
:104757004354435353203136352E35202020202013
:104767004354435353203136372E392020202020FD
:104777004354435353203137312E332020202020F8
:104787004354435353203137332E382020202020E1
:104797004354435353203137372E332020202020D2
:1047A7004354435353203137392E392020202020BA
:1047B7004354435353203138332E352020202020B3
:1047C7004354435353203138362E322020202020A3
:1047D7004354435353203138392E39202020202089
:1047E7004354435353203139322E38202020202080
:1047F7004354435353203139362E3620202020206E
:104807004354435353203139392E3520202020205B
:104817004354435353203230332E35202020202059
:104827004354435353203230362E35202020202046
:104837004354435353203231302E37202020202039
:104847004354435353203231382E31202020202027
:104857004354435353203232352E37202020202013
:104867004354435353203232392E31202020202005
:104877004354435353203233332E362020202020F5
:104887004354435353203234312E382020202020E4
:104897004354435353203235302E332020202020D9
:1048A7004354435353203235342E312020202020C7
:1048B70020202020202020202020202020202020F1
:1048C70044313233343536373839302A234142437D
:107B6B0075840F12553F12B4AB9000A8E0FF60056F
:107B7B00D3941440069000A87401F0128ABC12A191
:107B8B003112A18D12B3A5125389129FB9125367EB
:107B9B00123D28900118E0FF78A5760008A607E4AF
:107BAB0090018BF090022EF090022DF0900239F0A4
:107BBB0090023EF0129DB7E4900241F0900011F05C
:107BCB00125379D2ACD2A830311D12B52112B4ABFD
:107BDB00128ABC12A13112A18D12B3A5C236C237C3
:107BEB00C23812387580E0120056127D9220A32CF9
:107BFB00303F12C23F787EE6540F9048C7939001F6
:107C0B008AF01295AE3040E5C240787CE6540F9076
:107C1B0048C793900189F01296A480D120A4051235
:107C2B009EEF80F81288A9304126C24112B521126D
:107C3B00B4AB128ABC12A13112A18D12B3A5C236FC
:107C4B00C237C238129FB9E490022DF090022EF089
:107C5B00203606203703303805127DA480F243E727
:107C6B0040900013E0700E305508129F5612B54825
:107C7B0080031290D61279201249BB1276CB12B721
:037C8B0096809947
:105A50008DB7948A98419BDC9F3AA27EA5A9A8BAEB
:105A6000ABB1AEA5B150B40DB614B800BA6FBCD688
:105A7000BF14C148C365C577C74FC95FCB41CD0BC4
:105A8000CEC1D072D20DD2F2D39CD47FD51ED5F820
:105A9000D693D764D7FAD8C3D955DA16DAA8DB611A
:105AA000DBE9DC9FDD22DDD4DEFDE019E093E12EB1
:105AB000E239E33CE3AA000000000000000000001F
:105AC00000000000000000000000000000000000D6
:105AD00000000000000000000000000000000000C6
:105AE00000000000000000010000000000010000B4
:105AF00000000001000000000000000100000000A4
:105B00000001000000000001000000000001000092
:105B10000000000100000000000100000000000182
:105B20000000000000010000000000010000000172
:105B30000001000000010001000000010001000060
:105B40000001000100000000000100010000000150
:105B50000001000000010001000000010001000040
:105B6000000100010000000100010000000100012F
:105B70000000000100010000000100010000000120
:105B80000001000000010001000000010001000010
:105B900000010001000000010001000000010001FF
:105BA00000000001000100000001000100000001F0
:105BB00000010000000100010000000100010000E0
:105BC00000010001000000010001000100010001CE
:105BD00000010001000100010001000100010001BD
:0E5BE0000001000100010001000100010001B0
:10962900C22BC22DD2B3D2B275F006EFA424B6F57F
:1096390082E5F0345AF583E493FC740193FDEC4D13
:1096490024FF92B075F006EFA424B8F582E5F03452
:109659005AF583E493FC740193FDEC4D24FF92B712
:1096690075F006EFA424BAF582E5F0345AF583E4DF
:1096790093FC740193FDEC4D24FF92B5EF25E02492
:1096890050F582E4345AF583E493F52E740193F589
:0B9699002FD22CE4F584D28CD2A92241
:0EB7F100C22BC22DC22CE4F584C28CC2A92248
:104F0B0020504C55472050484F4E454C494E45205C
:104F1B0000554E504C55472050484F4E454C494E2E
:104F2B004500504C5547494E2050484F4E454C4933
:104F3B004E450044313233343536373839302A2335
:104F4B0041424302AB055508000AAB0D5510001248
:104F5B00AB155518001AAB1D55200022AB25552853
:104F6B00002AAB2D55300032AA355520205445531D
:104F7B005420524F5554494E45202020205645521F
:104F8B0053494F4E20312E3020202020544553546E
:104F9B00494E4720454550524F4D202020544553F4
:104FAB0054494E4720564F494345202054455354AE
:104FBB00494E472044544D462031202054455354EC
:104FCB00494E472044544D4620322020205445530F
:104FDB0054494E47205253323332202020544553EC
:104FEB0054494E4720525334383520202020544505
:104FFB005354494E47205054542020205445535469
:10500B00204155582052454C41592020544553546A
:10501B002043542052454C4159202020544553499C
:10502B004E472052494E47494E47202020202020F2
:10503B0020202020202020202020202054455354A5
:10504B00204C494E45204C4F4F5020544553542033
:10505B004C494E452053454E53452B5445535420F4
:10506B004C494E452053454E53452D5445535420E2
:10507B004C494E4520494E205553452054455354D9
:10508B0020494E50555420564F4C542054455354A0
:10509B00204C494E452052454C41595445535420C0
:1050AB005A45524F2043524F535320544553544962
:1050BB004E4720535155454C4348202020544553CF
:1050CB0054494E47204850462020202054455354E5
:1050DB002054454C434F20564F5820205445535491
:1050EB0020524144494F20564F5820202020202049
:1050FB0020202020202020202020202020202020A5
:10510B002020202020202020202020202020202094
:10511B0020202020202020202020202054455354C4
:10512B0020434F4D504C455445442020202054459E
:0B513B005354204641494C45442020BD
:103875007BFF7A4F797612ABEC7BFF7A4F79861214
:10388500A61212B8377BFF7A4F799612ABEC127DF0
:103895009212B837E4FFFE1275D3900170EFF07DF8
:1038A500AAE4FFFE127592E4FFFE1275D3EF64AA37
:1038B500600C7BFF7A51793612A6121200717D5584
:1038C500E4FFFE127592E4FFFE1275D3EF645560B6
:1038D5000C7BFF7A51793612A61212007190017095
:1038E500E0FDE4FFFE1275927BFF7A51792612AB5B
:1038F500EC12B8377BFF7A4F79A612ABEC125381E5
:1039050012B821E4F559755A01789E7614125D9C1A
:10391500789EE670FB125D9312B84BE4F559755A23
:1039250001789E7605789EE670FBD202D20B125D79
:103935008AC202C20B7BFF7A51792612ABEC12B810
:10394500377BFF7A4F79B612ABEC127D9212B837FE
:10395500C2277F3112B69E789E761E789EE670FB52
:1039650012B8523027FD787EE6547F904F3E937B08
:10397500FFB4310C7A51792612ABEC12B837800AB4
:103985007A51793612A6121200717BFF7A4F79C6E9
:1039950012ABEC127D9212B8377F3112B68712B88E
:1039A5004112B8523025FD787CE6547F904F3E9306
:1039B5007BFFB4310C7A51792612ABEC12B8378003
:1039C5000A7A51793612A6121200717BFF7A4F7965
:1039D500D612ABEC127D9212B837E4F58475985087
:1039E500C299C2987599433098FDE4F584E59964C8
:1039F50043600C7BFF7A51793612A6121200717B57
:103A0500FF7A51792612ABEC12B8377BFF7A4F79E2
:103A1500E612ABEC127D9212B83712538CE4F584A2
:103A2500759850C299C2987599433099FD7BFF7A74
:103A350051792612ABEC12B8377BFF7A4F79F61223
:103A4500ABEC127D9212B83712536112B841E532D0
:103A5500D39432400C7BFF7A51793612A6121200AC
:103A65007112536712B841E532C394AA500C7BFF1B
:103A75007A51793612A6121200717BFF7A51792696
:103A850012ABEC12B8377BFF7A50790612ABEC1209
:103A95007D9212B83712536D12B841E531D3940AAD
:103AA500400C7BFF7A51793612A61212007112531F
:103AB5007312B841E531C394AA500C7BFF7A517952
:103AC5003612A6121200717BFF7A51792612ABECE1
:103AD50012B8377BFF7A50792612ABEC127D921221
:103AE500B8371253A440FB7BFF7A51792612ABEC11
:103AF50012B8377BFF7A50794612ABEC127D9212E1
:103B0500B83712537912B8411253B0501A1253B63E
:103B150040157BFF7A50795612ABEC1253B040FB3F
:103B25001253B650F6801D1253B050DC1253B640F6
:103B3500D77BFF7A50796612ABEC1253B040FB127B
:103B450053B650F67BFF7A51792612ABEC12B83793
:103B55001253817BFF7A50797612ABEC127D92126B
:103B6500B8371253811253AA50107BFF7A4F790B45
:103B750012A6121253AA40FB800E7BFF7A4F791CC6
:103B850012A6121253AA50FB127D927BFF7A51792D
:103B95002612ABEC12B8371253817BFF7A50798627
:103BA50012ABEC127D9212B837E530C3940A400788
:103BB500E530D3943C400C7BFF7A51793612A6123E
:103BC5001200717BFF7A51792612ABEC12B8377B64
:103BD500FF7A50799612ABEC127D9212B8371253D8
:103BE5007912B84112539B400B7BFF7A4F792D1206
:103BF500ABEC80F07BFF7A51792612ABEC12B8372B
:103C05001253817BFF7A5079A612ABEC127D92128A
:103C1500B83712B80B1253A140FB1253A150FB1237
:103C250053A140FB7BFF7A51792612ABEC12B837D2
:103C350012B84B7BFF7A5079B612ABEC127D92121B
:103C4500B83712538F400B12536112536712538FBB
:103C550050F57BFF7A51792612ABEC12B8377BFF12
:103C65007A5079E612ABEC127D9212B83712B8167B
:103C750012539550FB12B84B7BFF7A51792612AB44
:103C8500EC12B8377BFF7A5079C612ABEC127D92F5
:103C950012B83712B80B12B739904F5012B730908F
:103CA5004F5212B730904F5412B730904F5612B74B
:103CB50030904F5812B730904F5A12B730904F5C32
:103CC50012B730904F5E12B730904F6012B73090F8
:103CD5004F6212B730904F6412B730904F6612B7EB
:103CE50030904F6812B730904F6A12B730904F6CD2
:103CF50012B730904F6E12B730904F7012B73090A8
:103D05004F7212B730904F74E493F508740193F530
:103D15000912B84B7BFF7A51792612ABEC12B837F2
:033D2500023C98C5
:0AB83700789E760A789EE670FB22E8
:0AB84100789E7602789EE670FB22E6
:09B73000E493F508740193F50996
:0AB73900789E7605789EE670FB22EC
:0200710080FE0F
:0300A30002A9A30C
:10A9A300C0E0C0F0C083C082C0D075D000C000C07A
:10A9B30001C002C003C004C005C006C0072055057E
:10A9C30012832A800312A4FCD007D006D005D0043A
:10A9D300D003D002D001D000D0D0D082D083D0F029
:03A9E300D0E0328F
:03009300029C7953
:099C7900C0E0C0D075D000C007A6
:109C8200AF84758402E543700885BE3375BB0780D7
:109C920032E543B4010885BE3075BB048025E54337
:109CA200B4020885BE3375BB068018E543B40308C9
:109CB20085BE3175BB04800BE543B4040A85BE330F
:109CC20075BB0505438010E543B4050885BE3275B2
:0B9CD200BB048000754300C2ED8F84CE
:079CDD00D007D0D0D0E03227
:0300830002AC24A8
:10AC2400C0E0C0F0C083C082C0D075D000C000C0F6
:10AC340001C002C003C004C005C006C007C2CF12D1
:10AC44001700D007D006D005D004D003D002D0011D
:0DAC5400D000D0D0D082D083D0F0D0E0323C
:03007B0002A07868
:10A07800C0E0C0F0C083C082C0D075D000C000C0AE
:10A0880001C002C003C004C005C006C00720240FD9
:10A0980085BF4085BE3FD22475BB01C2ED801385C4
:10A0A800BF3E85BE3DC22430580312817175BB0086
:10A0B800C2EDD007D006D005D004D003D002D0011D
:0DA0C800D000D0D0D082D083D0F0D0E032D4
:03007300028FAF4A
:108FAF00C0E0C0F0C083C082C0D075D000C000C088
:108FBF0001C002C003C004C005C006C007C2CF78FD
:108FCF009AE6600116302E27124C1EC22ED55C0574
:108FDF00755C0A055BD51B09751B0A7584014388EF
:108FEF0020D51C19751C60758402438820800ED211
:108FFF002E789B16E670067604F584D28B305505D5
:10900F00129E20800312A3A712928312980F7584C9
:10901F0001438810758400D2ECD007D006D005D05C
:10902F0004D003D002D001D000D0D0D082D083D0D2
:04903F00F0D0E0325B
:03006B000287E920
:1087E900C0E0C0F0C083C082C0D075D000C000C056
:0D87F90001C002C003C004C005C006C007D7
:1088060085841620261875840F30DF3875840FE5A9
:10881600E8540F787CF6D226787D76C88026787D57
:1088260016E6700E75840FE5E8540F787CF6E6447C
:1088360080F675840F20DF0CC226D225D240D26284
:10884600D25FD26820281630F833E5E854F0FFC42A
:10885600540F787EF6D228787F76C88020787F16E7
:10886600E6700FE5E854F0FFC4540F787EF6E64450
:1088760080F620F808C228D227D23FD2611274525D
:08888600758402C28D85168481
:10888E00D007D006D005D004D003D002D001D0003E
:0B889E00D0D0D082D083D0F0D0E032E8
:03005B0002A1E916
:10A1E900C0E0C0F0C083C082C0D075D000C000C03C
:10A1F90001C002C003C004C005C006C0071248F070
:10A20900789CE6600116E5416002154190000CE07A
:10A21900600214F0900247E0600214F0758401C2F4
:10A229008DD007D006D005D004D003D002D001D0FC
:0CA2390000D0D0D082D083D0F0D0E03232
:0300530002A850B0
:10A85000C0E0C0F0C083C082C0D075D000C000C0CE
:10A8600001C002C003C004C005C006C007C28C30CE
:10A870005A04C25A8005D25A124D3DD007D006D094
:10A8800005D004D003D002D001D000D0D0D082D0E7
:06A8900083D0F0D0E0329D
:03002B0002000FC1
:03000F00C2CF322B
:03001B0002006E72
:03006E00C28F320C
:0300130002AE0238
:10AE0200C0E0C0F0C083C082C0D075D000C000C016
:10AE120001C002C003C004C005C006C0071213E887
:10AE2200D007D006D005D004D003D002D001D00084
:0BAE3200D0D0D082D083D0F0D0E0322E
:10AAA900191823A01296203D129623A01296276307
:10AAB9001488203D148823A01488276316B8203DE4
:10AAC90016B823A016B827631918203D191827634B
:10AAD90012962B8C14882B8C16B82B8C19182B8C4E
:0BB8210075081575095ED229D20322BC
:0BB82C0075081575095ED229D20C22A8
:07B84B00C229C203C20C2256
:10B68700E4F512F513F514F5159000F3E0F535120E
:07B697006F0BD22AD204223E
:10B69E00E4F512F513F514F5159000F4E0F53512F6
:07B6AE006F0BD22AD20D221E
:106F0B00EF127F7E7006236FF52A6F43306F55317A
